:100000000C9445080C946D080C946D080C94FA152A
:100010000C94FA150C94FA150C946D080C946D0858
:100020000C946D080C946D080C946D080C946D087C
:100030000C946D080C946D080C946D080C946D086C
:100040000C94B0150C946D080C94AF140C94891496
:100050000C946D080C946D080C946D080C946D084C
:100060000C946D080C946D0800000000060001005F
:100070000002120803EF050006060801F00A000D51
:10008000100D00F124000B140D01EF4000141115A8
:1000900001F06B000E111001F0890002060501F05D
:1000A0008B0005170802EF9A0005170801EFA90059
:1000B00007070901EFB0000A0B0E02F6BE000206A8
:1000C0000702FFC00006020801F9C2000202060290
:1000D000FFC30007120700EFD3000B110D01F0EB77
:1000E0000005110D03F0F6000B110D01F00E010BD0
:1000F000110D01F026010B110D01F03E010B110D48
:1001000001F056010B110D01F06E010B110D01F004
:1001100086010B110D01F09E010B110D01F0B601CE
:10012000020D0602F4BA0102100602F5BE010C0C23
:100130000E01F5D0010C060E01F8D9010C0C0E01D0
:10014000F5EB010A120D02EF020216151801EF3C41
:100150000210121000EF60020D121002EF7E020F6B
:10016000121101EFA0020E121102EFC0020C120FC9
:1001700002EFDB020B120E02EFF40210121201EF7B
:1001800018030D121102EF360302120702EF3B03B0
:1001900009120D01EF50030E121002EF70030A1244
:1001A0000E02EF870310121402EFAB030D121202BE
:1001B000EFC90311121301EFF0030C121002EF0B41
:1001C0000411131301EF34040E121102EF54040E44
:1001D000121001EF74040C120F01EF8F040D1211B5
:1001E00002EFAD040F120F00EFCF0416121600EF4E
:1001F00001050F121000EF230510121000EF470544
:100200000D120F01EF650504170702EF71050712C4
:100210000700EF810504170701EF8D0509090B01A0
:10022000F098050F010DFF049A0505040601EF9DE6
:10023000050C0D0D01F4B1050C120D01EFCC050AF2
:100240000D0C01F4DD050B120D01EFF6050B0D0D84
:1002500001F4080605120701EF14060B120D01F454
:100260002D060A120D01EF440602120502EF49069F
:1002700004170600EF55060B120C01EF6E06021272
:100280000501EF7306110D1301F48F060A0D0D0120
:10029000F4A0060B0D0D01F4B2060C110D01F4CC07
:1002A000060B110D01F4E406060D0801F4EE060A32
:1002B0000D0C01F4FF0605100701F109070A0D0DE9
:1002C00001F41A070C0D0C00F42E07110D1100F4A7
:1002D0004A070B0D0B00F45C070B120B00F47507BB
:1002E0000A0D0C01F4860705170801EF95070217A0
:1002F0000602EF9B0705170802EFAA070A050C0183
:10030000F6FFFFFFF0F0CF3CF38A200630310318F0
:1003100018C7FFBFFC31031818C7FFBFFC31011815
:1003200018C0C606300403E1FF726C4788F107204D
:100330007E03F017023C4788F11B267FC3E01002C2
:1003400000000603C0407E0C0E7080C3180C310004
:10035000E73007E6003C40000C7C008FE019C70145
:1003600018303183021C7040FE0407C00F007E036A
:100370009C0C3030C0E701F803803E01CC6E19B010
:100380007CC0F303CE1F9FE61E1CFFA0088C6631C5
:1003900098C6318C63086308610C208218C318C3A7
:1003A00018C6318C623188C4620010235BE38D91E2
:1003B000000C0300C030FFFFF0C0300C0300C0F59C
:1003C00060FFF0F0020C1020C1020C1020C1020CE2
:1003D0001020C1001F07F1C7306E0F80F01E03C050
:1003E000780F01E03C0EC19C71FC1F0008CFFF8C10
:1003F0006318C6318C63181F0FF987607C0600C034
:10040000180701C0F0781C0600803007FFFFE03FAE
:100410000FF387606C0C0180707C0F801801803CAA
:100420000780D873FC1F000180700E03C0D81B0624
:10043000618C218C33067FFFFE0300600C01803F3E
:10044000CFF980300600DE1FE70E00E00C0180309F
:100450000781F873FC1F000F07F9C3307401803364
:10046000C7FEF0DC1F01E03C06C1DC71FC1F00FF91
:10047000FFFC010060180200C0300601803004015A
:10048000803006018030001F07F1C730660CC18C38
:1004900061FC3F8E3B01E03C0780D831FC1F001F10
:1004A00007F1C7706C0780F01E0761EFFC798030A0
:1004B00005819873FC1E00F00003C0F0000F560089
:1004C000000701E0F83C0F00E007C00F003C00F01F
:1004D00001FFFFFF000000FFFFFF000E007801F0AA
:1004E00007C00F00701E0F03C0F008001F1FEE1B97
:1004F00003C0C0300C060381C0E0300C03000000D4
:100500000C030000FE000FFE00F03E07003C380028
:1005100030C1E0660FD9D861C3C3070F1C1C3C6013
:1005200060F18183C6061B1838EE71E718FDF8717B
:10053000E7C0E00001E00001FFC001FC0003C003D0
:10054000C003C007E0066006600E700C300C301C63
:100550003818181FF83FFC301C300C700E60066015
:1005600006FFC7FF3019806C03601B00D80CFFC763
:10057000FF300D803C01E00F007806FFF7FE00071A
:10058000E03FF0E0738066006C0030006000C00166
:10059000800300060006006C00DC031E0E1FF80F2F
:1005A000C0FF83FF8C07300EC01B007C00F003C02F
:1005B0000F003C00F003C01F006C03B01CFFE3FF02
:1005C00000FFFFFFC00C00C00C00C00C00FFEFFEDE
:1005D000C00C00C00C00C00C00FFFFFFFFFFFF00BD
:1005E000600C0180300600FFDFFB00600C018030F2
:1005F0000600C0180007F01FFC3C1E70066003E0F8
:1006000000C000C000C07FC07FC003C003600360A3
:1006100007300F3C1F1FFB07E1C01E00F007803CA6
:1006200001E00F007803FFFFFFF007803C01E00FBF
:10063000007803C01E00C0FFFFFFFFF00180C06014
:1006400030180C06030180C0603C1E0F07C77F1FD7
:1006500000C03B01CC0E3070C3831C0CE03380DE45
:1006600003DC0E383060C1C3038C06301CC03B0075
:1006700060C0300C0300C0300C0300C0300C03001D
:10068000C0300C0300FFFFF0E007E007F00FF00FB1
:10069000D00FD81BD81BD81BCC33CC33CC33C6637C
:1006A000C663C663C3C3C3C3C3C3C183E01F00FC27
:1006B00007E03D81EE0F3079C3C61E18F0E7833C9A
:1006C0001DE06F01F80FC03E01C003E00FFC0F07F3
:1006D0008600C60033001B00078003C001E000F065
:1006E0000078003600330018C018783C1FFC03F86F
:1006F00000FF8FFEC06C03C03C03C03C07FFEFFC53
:10070000C00C00C00C00C00C00C00C0003E00FFCCB
:100710000F078600C60033001B00078003C001E0FE
:1007200000F00078003600330198C0FC783C1FFFD1
:1007300003F9800040FFC3FFCC03B006C01B006C70
:1007400001B00CFFE3FFCC03B006C01B006C01B08E
:1007500006C01B00700FE07FC3839C07600D8006FE
:10076000001E003F803FC00F8007C00F003E00DE2C
:100770000E3FF03F80FFFFFF0600600600600600AE
:10078000600600600600600600600600600600600B
:10079000C01E00F007803C01E00F007803C01E007F
:1007A000F007803C01E00F80EE0E3FE07C00600629
:1007B000C01DC031806301C70306060C1C1C301825
:1007C0006031C073006600DC01F001E003C0070087
:1007D000E0301D80E0760781D81E06707C18C1B01D
:1007E000E30CC38C330C38C6306718C198670661B8
:1007F000D81D83603C0D80F03E03C0700F01C0180F
:100800000700700E6038E060E1C0C301CC01F80160
:10081000E0038007801F003300E70386060E1C0EEE
:10082000700CC01C6006700E301C38181C380C3060
:100830000E70066003C003C001800180018001804A
:100840000180018001800180FFFFFFC00E00E00EEB
:10085000006007007007003003803803801801C073
:100860001C00FFFFFFC0FFCCCCCCCCCCCCCCCCCC84
:10087000CFF08181020604081810206040818102B7
:100880000604FF3333333333333333333FF00C0E4B
:100890000586C321198C83C180FFFEE38C303F079E
:1008A000F8E1CC0C00C01C3FCF8CC0CC0CE3C7EFF0
:1008B0003C70C00C00C00C00C00CF8DFCF0EE07C18
:1008C00003C03C03C03C03E06F0EDFCCF81F0FE712
:1008D0001B83C0300C0300C038371CFE1F000060B3
:1008E0000C018030063CCFFB8FE0F80F01E03C07A5
:1008F00080F83B8F3F63CC1F07F1C7703C07FFFFB9
:10090000FE00C01C0DC31FE1F03BD8C67FEC63188E
:10091000C6318C63001E67FDC7F07C0780F01E03A4
:10092000C07C1DC79FB1E600C03E0E7FC7E0C0304F
:100930000C0300C033CDFBC7E0F03C0F03C0F03C1C
:100940000F03C0F030F03FFFFFF0330003333333C9
:10095000333333333FE0C0180300600C018330C6EB
:1009600030CC1B83F0770C618E30E60CC1D818FFB9
:10097000FFFFFFF0CF1F6FDFFC78FC183C0C1E065A
:100980000F03078183C0C1E060F03078183C0C1879
:10099000CF37EF1F83C0F03C0F03C0F03C0F03C004
:1009A000C01F07F1C7707C0780F01E03C07C1DC705
:1009B0001FC1F0CF8DFCF0EE06C03C03C03C03C06D
:1009C0003E07F0EFFCCF8C00C00C00C0001E67FD9E
:1009D000C7F07C0780F01E03C07C1DC79FF1E600B6
:1009E000C018030060CF7F38C30C30C30C30C03E4A
:1009F0001FEE1B00C03C07F03E01F03E1DFE3E0016
:100A00006319FFB18C6318C631E7C0F03C0F03C017
:100A1000F03C0F03C0F07E3DFB3CC0E06606606723
:100A20000C30C30C3981981981F00F00E00E00C121
:100A3000C1B0E1D870CC2C6636319B18CD98646C6F
:100A400016360F1A078F038380C1C060EE18C60CDC
:100A5000C1F01C0180781B0330C7306606E06C0DC6
:100A60008338630C630E60CC1B03603C0700E01806
:100A70000300E0780E00FFFFF0180C070381C06050
:100A800030180E03FFFFC019CC6318C631998618C1
:100A9000C6318C631C60FFFFFFFFFFFCC718C63127
:100AA0008C630C33318C6318C67300703E09E41FED
:100AB000038001036800207E1D04E010021C071261
:100AC0003732292D29252B3900010310E110031D90
:100AD00007062E2C292D2E2E373F000002101380E2
:100AE0000A298064022A040000007F2B0400000011
:100AF0009F0F0180961180FFB103012C2DB20301DD
:100B00002C2DB306012C2D012C2DB40107C003A2FE
:100B10000284C101C5C2020A00C3028A2AC4028A31
:100B2000EEC5010E20003601C83A010500000000A4
:100B3000003E5B4F5B3E3E6B4F6B3E1C3E7C3E1C63
:100B4000183C7E3C181C577D571C1C5E7F5E1C00A9
:100B5000183C1800FFE7C3E7FF0018241800FFE760
:100B6000DBE7FF30483A060E2629792926407F0523
:100B70000507407F05253F5A3CE73C5A7F3E1C1C39
:100B800008081C1C3E7F14227F22145F5F005F5FF9
:100B900006097F017F006689956A606060606094E5
:100BA000A2FFA29408047E040810207E20100808EA
:100BB0002A1C08081C2A08081E101010100C1E0CF5
:100BC0001E0C30383E3830060E3E0E060000000087
:100BD0000000005F00000007000700147F147F146E
:100BE000242A7F2A122313086462364956205000B3
:100BF00008070300001C2241000041221C002A1C9F
:100C00007F1C2A08083E0808008070300008080889
:100C10000808000060600020100804023E514945A9
:100C20003E00427F400072494949462141494D33C7
:100C30001814127F1027454545393C4A494931412E
:100C4000211109073649494936464949291E0000FC
:100C50001400000040340000000814224114141451
:100C60001414004122140802015909063E415D593D
:100C70004E7C1211127C7F494949363E4141412246
:100C80007F4141413E7F494949417F090909013E70
:100C9000414151737F0808087F00417F4100204097
:100CA000413F017F081422417F404040407F021CA9
:100CB000027F7F0408107F3E4141413E7F090909C0
:100CC000063E4151215E7F0919294626494949328C
:100CD00003017F01033F4040403F1F2040201F3F52
:100CE0004038403F631408146303047804036159D7
:100CF000494D43007F414141020408102000414119
:100D0000417F0402010204404040404000030708C4
:100D10000020545478407F284444383844444428C0
:100D2000384444287F385454541800087E09021867
:100D3000A4A49C787F0804047800447D40002040EF
:100D4000403D007F1028440000417F40007C047833
:100D500004787C080404783844444438FC1824247B
:100D60001818242418FC7C080404084854545424FB
:100D700004043F44243C4040207C1C2040201C3C78
:100D80004030403C44281028444C9090907C44646F
:100D9000544C440008364100000077000000413602
:100DA000080002010204023C2623263C1EA1A16188
:100DB000123A4040207A38545455592155557941BA
:100DC0002254547842215554784020545579400C8F
:100DD0001E52721239555555593954545459395572
:100DE0005454580000457C410002457D42000145B5
:100DF0007C407D1211127DF0282528F07C54554549
:100E0000002054547C547C0A097F493249494932B4
:100E10003A4444443A324A4848303A4141217A3AC5
:100E200042402078009DA0A07D3D4242423D3D4091
:100E300040403D3C24FF2424487E4943662B2FFC40
:100E40002F2BFF0929F620C0887E090320545479EE
:100E5000410000447D413048484A32384040227ABF
:100E6000007A0A0A727D0D19317D2629292F28263C
:100E70002929292630484D40203808080808080844
:100E80000808382F10C8ACBA2F102834FA00007B9D
:100E9000000008142A142222142A140855005500B0
:100EA00055AA55AA55AAFF55FF55FF000000FF009F
:100EB000101010FF00141414FF001010FF00FF109A
:100EC00010F010F0141414FC001414F700FF0000CC
:100ED000FF00FF1414F404FC141417101F10101F4B
:100EE000101F1414141F00101010F0000000001F39
:100EF000101010101F10101010F010000000FF1044
:100F00001010101010101010FF10000000FF14003F
:100F100000FF00FF00001F10170000FC04F4141471
:100F20001710171414F404F40000FF00F71414143D
:100F300014141414F700F7141414171410101F10BD
:100F40001F141414F4141010F010F000001F101FE0
:100F50000000001F14000000FC140000F010F0104E
:100F600010FF10FF141414FF141010101F000000C5
:100F700000F010FFFFFFFFFFF0F0F0F0F0FFFFFFC9
:100F80000000000000FFFF0F0F0F0F0F3844443820
:100F900044FC4A4A4A347E02020606027E027E026F
:100FA00063554941633844443C04407E201E20067A
:100FB000027E020299A5E7A5991C2A492A1C4C72B7
:100FC00001724C304A4D4D303048784830BC625A3E
:100FD000463D3E494949007E0101017E2A2A2A2ACE
:100FE0002A44445F444440514A444040444A5140AA
:100FF0000000FF0103E080FF000008086B6B08366B
:1010000012362436060F090F0600001818000000DB
:101010001010003040FF0101001F01011E00191DCA
:101020001712003C3C3C3C000000000000000000A7
:10103000240027002A00000000080002010000032D
:101040000407000000000000000000000000250070
:1010500028002B00000000002300260029000404C3
:101060000404040404040202020202020303030350
:10107000030301020408102040800102040810202C
:1010800001020408102059314F3111241FBECFEF47
:10109000D8E0DEBFCDBF13E0A0E0B1E0EEE2F2E7C2
:1010A00002C005900D92A632B107D9F724E0A6E25E
:1010B000B3E001C01D92A839B207E1F718E0C4E41B
:1010C000D8E004C02197FE010E94FF38C334D10745
:1010D000C9F70E948C1C0C940A390C9400000895E6
:1010E000FC016370658B8481958126813781613035
:1010F00039F0633029F091878087338722870895FC
:10110000318720879387828708952F923F924F924D
:101110005F926F927F928F929F92AF92BF92CF9287
:10112000DF92EF92FF920F931F93CF93DF93CDB790
:10113000DEB76C970FB6F894DEBF0FBECDBF9C8FA5
:101140008B8F5B011A011F830E833701C982DC017B
:1011500058964D915C9159974115510509F0E5C09C
:1011600018968D919C911997681779070CF0CAC150
:101170001A968D919C911B97281639060CF0C2C1C6
:101180008C2C912CFB0136E0C39EE00DF11D112447
:10119000FB87EA871E161F060CF0B4C1C40133E0BA
:1011A000880F991F3A95E1F79D878C87820D931DD3
:1011B000181619060CF0A6C157968C91811103C020
:1011C000203B08F02F5FAB8DBC8DED91FC9111970A
:1011D0000284F385E02DCD012A8F09952A8DB5E093
:1011E0002B9F90011124F5013596FF87EE87BB8276
:1011F000AA822501A9014A195B09598B488BC101B3
:1012000008969B8B8A8BE889F989E40DF51DE45DCE
:10121000F44F9491988761013D822C82A885A0FFAC
:1012200013C0AB8DBC8DED91FC91B981B13031F41F
:101230000484F585E02D2E813F8116C00684F78554
:10124000E02DEE80FF801AC0EE81FF816E167F06D2
:10125000F1F0AB8DBC8DED91FC91B981B13051F4C1
:101260000484F585E02D9301A601B2018B8D9C8D40
:1012700009950DC00684F785E02D73018401940162
:101280004C815D816A817B818B8D9C8D0995E88580
:10129000E695E887FFEFCF1ADF0A2C813D81280D04
:1012A000391D3D832C834A895B89C416D50609F014
:1012B000B5CF5FEF451A550A8A819B81880D991D2C
:1012C0009B838A83AE85BF854A165B0609F09BCF58
:1012D000EE81FF816E167F0609F4F2C0EB8DFC8D66
:1012E000A081B181F981F13079F4B5016B5F7F4F55
:1012F0005096ED91FC915197830128E030E0A101D7
:101300008B8D9C8D0995DCC06A857B856819790970
:101310001E96ED91FC911F9773010C851D8594011C
:10132000A1018B8D9C8D0995CBC0FA0134969491C7
:10133000329765917491291BCB01B7E02B9F800DEB
:10134000911D1124FA01259134913B8B2A8BFC01CC
:10135000459154915B834A83FC013296C490319647
:1013600054915E87329614913196D490898182305F
:1013700058F0612E012E000C7708AD2D0D2C000CBD
:10138000BB0BB987A88704C019861886612C712CFD
:10139000AB8DBC8DED91FC9111970284F385E02D0E
:1013A000CD010995B9818B2E912C689CC001699C57
:1013B000900D789C900D1124FC01EA0DFB1DFD871A
:1013C000EC871C82712C612CE12F110FFF0B950112
:1013D0002E0F3F1F3B872A87AC0CB11CA5014E0F77
:1013E0005F1F5F8B4E8BC1018D0D911DD7FC9A95B0
:1013F000998F888F4E85641608F062C0862D90E024
:1014000048855985480F591F489D9001499D300DC9
:10141000589D300D1124D901A20DB31DB98BA88B95
:10142000AA84BB844C845D84DC80BA85DB1AE88D99
:10143000F98DE80FF91FFD8BEC8B8D2D8A0D2E8910
:101440003F89A216B306B9F1877061F48A819B8146
:101450000196EA89FB89AA81BB81EA0FFB1F749080
:101460009B838A8377FE20C0AB8DBC8DED91FC9170
:10147000B981B13061F40484F585E02D2E813F817E
:101480004C895D89B5018B8D9C8D09950DC00684B5
:10149000F785E02DEE80FF80840194014889598909
:1014A000B2018B8D9C8D0995770CEFEFAE1ABE0AB9
:1014B000480C591CC2CF3C813C0D3C8363949ACFAD
:1014C000AB8DBC8DED91FC9111970688F789E02DCD
:1014D000CD016C960FB6F894DEBF0FBECDBFDF9185
:1014E000CF911F910F91FF90EF90DF90CF90BF9021
:1014F000AF909F908F907F906F905F904F903F90B4
:101500002F9009946C960FB6F894DEBF0FBECDBF36
:10151000DF91CF911F910F91FF90EF90DF90CF90CF
:10152000BF90AF909F908F907F906F905F904F9003
:101530003F902F900895AF92BF92CF92EF92FF927B
:101540000F931F93CF93DF93EC01262F888D998DF6
:10155000009709F040C06A3059F41D861C862C891A
:101560008E859F8538E0239F800D911D112441C0F9
:101570006D3009F4AAC08E898823C1F03C898C851E
:101580009D8546E0349F800D911D11244885598525
:10159000481759075CF41D861C868E859F8548E098
:1015A000349F800D911D11249F878E87EA88FB88C8
:1015B000088919894E855F856C857D85CC88CE012B
:1015C0000E9485082C898C859D8536E0239F800D9F
:1015D000911D112442C06A3079F41D861C862C8925
:1015E000FC013696E4918E859F852E9F800D911D7E
:1015F00011249F878E8769C06D3009F466C0FC0195
:1016000034963491631708F460C03196E491E6177C
:1016100008F45BC0FC013296A590B490462F50E0D0
:10162000431B510937E0349FB001359F700D1124E1
:10163000A60EB71EF501329634913196E49133230C
:1016400011F0E1110DC0F5013496E4912C898C85DF
:101650009D85E29F800D911D11249D878C8735C04B
:10166000F501359644915E89552311F16C89E32F7C
:10167000F0E0E40FF11D47FDFA956E9FD0016F9FDA
:10168000B00D11244C855D854A0F5B1FE885F985F7
:10169000E417F5076CF41D861C86FC013696E49170
:1016A0008E859F856E9F800D911D11249F878E874B
:1016B000EA88FB88088919894E855F856C857D8558
:1016C000CC88CE010E948508BECF81E090E0DF91FA
:1016D000CF911F910F91FF90EF90CF90BF90AF905F
:1016E00008956F927F928F929F92AF92BF92CF9206
:1016F000DF92EF92FF920F931F93CF93DF93EC0152
:101700004B015A0169013801E881F9810284F385AE
:10171000E02D0995E881F9810288F389E02D8701A0
:101720009601A501B401CE010995E881F981A501D1
:10173000460D571D415051090288F389E02D96014D
:10174000B401CE010995E881F9810088F189E02D85
:101750009301A501B401CE010995E881F981C80C76
:10176000D91CB601615071090088F189E02D9301FF
:10177000A501CE010995E881F9810688F789E02D58
:10178000CE01DF91CF911F910F91FF90EF90DF90ED
:10179000CF90BF90AF909F908F907F906F90099463
:1017A000CF92DF92EF92FF920F931F93CF93DF932D
:1017B00000D000D000D0CDB7DEB76C01DC01ED91D8
:1017C000FC916217730789F4041715072CF4942F02
:1017D000852FA801092F182F041B150B98012F5FC7
:1017E0003F4F048CF58DE02D12C04017510709F5CD
:1017F000261737072CF4962F872FB901292F382F5A
:10180000261B370B2F5F3F4F068CF78DE02D87018E
:10181000C601099526960FB6F894DEBF0FBECDBF60
:10182000DF91CF911F910F91FF90EF90DF90CF90BC
:1018300008950284F385E02D2D833E834B835C83E2
:1018400069837A830995D601ED91FC910488F58925
:10185000E02D2D813E814B815C8169817A81C601B9
:101860000995D601ED91FC910688F789E02DC60116
:1018700026960FB6F894DEBF0FBECDBFDF91CF9195
:101880001F910F91FF90EF90DF90CF900994EF920E
:10189000FF920F931F93DC01ED91FC9111971A9623
:1018A0000D911C911B9718962D913C91199700A0B2
:1018B000F1A1E02D7B0140E050E060E070E009958F
:1018C0001F910F91FF90EF9008954F925F926F924A
:1018D0007F928F929F92AF92BF92CF92DF92EF92C0
:1018E000FF920F931F93CF93DF9300D0CDB7DEB756
:1018F0006C015A0139014801DC01ED91FC9102842F
:10190000F385E02D69837A8309956981462E7A8172
:10191000572E640C751CD601ED91FC9146145704AA
:101920006CF40088F189E02D87019401A501B201D2
:10193000C6010995BFEF4B1A5B0AEDCF0688F78900
:10194000E02DC6010F900F90DF91CF911F910F9165
:10195000FF90EF90DF90CF90BF90AF909F908F90CF
:101960007F906F905F904F900994AF92BF92CF920B
:10197000DF92EF92FF920F931F93CF93DF9300D0EC
:1019800000D0CDB7DEB75C016901DC01ED91FC91BF
:101990000284F385E02D4B835C8369837A83099508
:1019A000D501ED91FC9169817A819B012C0D3D1D42
:1019B000215031090488F589E02D78014B815C8143
:1019C0008A01C5010995D501ED91FC910688F78939
:1019D000E02DC5010F900F900F900F90DF91CF91E8
:1019E0001F910F91FF90EF90DF90CF90BF90AF903D
:1019F0000994AF92BF92CF92DF92EF92FF920F9332
:101A00001F93CF93DF9300D000D0CDB7DEB75C013A
:101A10006901DC01ED91FC910284F385E02D4B839B
:101A20005C8369837A830995D501ED91FC914B81A3
:101A30005C81C40ED51EB1E0CB1AD1080488F589AB
:101A4000E02D7801860169817A819B01C5010995A4
:101A5000D501ED91FC910688F789E02DC5010F9025
:101A60000F900F900F90DF91CF911F910F91FF90EA
:101A7000EF90DF90CF90BF90AF9009940895EF92D0
:101A8000FF920F931F93DC01ED91FC9100A0F1A157
:101A9000E02D09951F910F91FF90EF9008950F93FE
:101AA0001F93DC01ED91FC91068CF78DE02D0995DB
:101AB0001F910F9108950F931F93DC01ED91FC91FD
:101AC000048CF58DE02D09951F910F910895DC018F
:101AD000ED91FC910084F185E02D099408952F92F9
:101AE0003F924F925F926F927F928F929F92AF92AE
:101AF000BF92CF92DF92EF92FF920F931F93CF93FB
:101B0000DF9300D01F92CDB7DEB74C017B836A8391
:101B10006A01590117019801241B350B37FF03C0D7
:101B2000319521953109C5014A815B81841B950B53
:101B300097FF03C091958195910951E059838217D0
:101B4000930714F019820BC09A2D8B2D5801092F81
:101B5000182F9A818B81DB82CA82C92ED82E8A8166
:101B60009B81A816B9065CF49C2D8D2D6801092F68
:101B7000182F9A818B81BB82AA82A92EB82E2501AB
:101B8000AA81BB814A1A5B0A38016C187D0877FE6E
:101B900003C0719461947108720157FE03C0BFEFD6
:101BA000EB1AFB0AF594E794C016D1061CF00FEF70
:101BB0001FEF1FC001E010E01CC0D401ED91FC91AB
:101BC000B9810484F585E02D9101BB23C1F04A81E0
:101BD0005B81B601C4010995E618F708F7FE04C059
:101BE000C00ED11EE40CF51CEA81FB813196FB830B
:101BF000EA834A815B81A416B506FCF604C0A601FF
:101C00006A817B81E7CF0F900F900F90DF91CF918A
:101C10001F910F91FF90EF90DF90CF90BF90AF900A
:101C20009F908F907F906F905F904F903F902F90FC
:101C30000895089580E090E0089508958CBD9DBDBD
:101C4000089589E794E00E9474160E94271A62E7BB
:101C500072E088EA93E00E9487146CEF89E794E0D1
:101C60000E94341362E070E080E090E00E947615FC
:101C70008FB7F89440912603509127036091280371
:101C8000709129038FBF4C505E4F6F4F7F4F409331
:101C90002A0350932B0360932C0370932D0388EA3F
:101CA00093E00E94F51961E472E088EA93E00C94F5
:101CB000151460E070E08AE494E00C94C1130F9373
:101CC0001F93CF93DF93109278041092770461E012
:101CD00080916F040E943A1561E080916E040E9429
:101CE0003A1520916E0430E0F901E25AFF4EE4917A
:101CF000F0E0EE0FFF1FE65BFF4E8591949190930D
:101D00006B0480936A0440916F0450E0FA01E25A38
:101D1000FF4E8491E82FF0E0EE0FFF1FE65BFF4ED1
:101D20008591949190936D0480936C04F901EE5821
:101D3000FF4EE491E0937504FA01EE58FF4EE491F2
:101D4000E093760480916504882309F43AC0CFB704
:101D5000F89480915803811127C0E8E6F0E184915E
:101D6000ECE7F0E19491E82FF0E0EE0FFF1FE45D67
:101D7000FF4EA591B491EC91E92321F461E08AE052
:101D80000E940A1561E08AE00E943A158CB58061D4
:101D90008CBD8CB580648CBD61E08DE00E943A15ED
:101DA00061E08BE00E943A15809158038F5F809329
:101DB0005803CFBF80E58093450481E080934604BB
:101DC00048C061E0809172040E943A1561E0809100
:101DD00071040E943A158091720490E0FC01E25A6D
:101DE000FF4EE491F0E0EE0FFF1FE65BFF4EA59182
:101DF000B491B0936904A09368042091710430E019
:101E0000F901E25AFF4EE491F0E0EE0FFF1FE65BAE
:101E1000FF4E459154915093670440936604FC0132
:101E2000EE58FF4E849180937404F901EE58FF4EF2
:101E3000E491E0937304EC9180958E238C93E09170
:101E40006604F091670490818091730480958923E2
:101E50008083E0916A04F0916B0490818091750415
:101E600080958923808380917004882321F161E02B
:101E70000E943A1561E0809170040E940A1564EF97
:101E800071E080E090E00E94761560E0809170043F
:101E90000E940A1564EF71E080E090E00E947615E0
:101EA00061E0809170040E940A1564EF71E080E0A7
:101EB00090E00E94761581EF9AE00E94431B84EE29
:101EC0009AE00E94431B89EB9AE00E94431B66E361
:101ED0008AE494E00E94C31660EC8AE494E00E94D5
:101EE0008A1682E0809364048091490490E00E9405
:101EF000E91A60E070E08AE494E00E94C11363E0B4
:101F00008AE494E00E94041782EB9AE00E94C91AC6
:101F100081E080935E0486E190E090935704809383
:101F200056048CE190E0909359048093580480EE1D
:101F30009FEF90935D0480935C0490935B04809387
:101F40005A0460E872E08AE494E00E94871487E112
:101F500090E090935704809356040DE110E01093A5
:101F6000590400935804C0E0D8EFD0935D04C093A7
:101F70005C04D0935B04C0935A0460E872E08AE486
:101F800094E00E94871488E190E090935704809336
:101F900056041093590400935804D0935D04C093E1
:101FA0005C04D0935B04C0935A0460E872E08AE456
:101FB00094E00E94871468EE73E080E090E00E9455
:101FC000761589E794E00E9474160E94271A6BE840
:101FD00072E088EA93E00E9473146FEF89E794E05F
:101FE0000E94341364E170E080E090E00E94761576
:101FF00089E794E00E948813892B09F440C089E79F
:1020000094E00E94A013EC0167E972E088EA93E093
:102010000E948714AE010D2E000C660B770B88EA28
:1020200093E00E94F51962E070E080E090E00E9489
:10203000761520912F03309130032115310529F4B5
:10204000D0935C03C0935B0313C02130310529F4A6
:10205000D0935E03C0935D030BC02330310519F4A8
:10206000C0935A0305C02430310511F4C0935903BD
:102070002F5F3F4F3093300320932F03B9CF10923F
:10208000300310922F0380E090E00E94C91A83E48D
:1020900090E090935704809356048CE390E09093E3
:1020A00059048093580480EE9FEF90935D048093D1
:1020B0005C0490935B0480935A0481E080935E04F7
:1020C00080915D0390915E03892B31F46CE972E09D
:1020D0008AE494E00E94871480915D0390915E03EE
:1020E000019731F463EA72E08AE494E00E94871475
:1020F00080915D0390915E03029731F467EA72E08C
:102100008AE494E00E94871480915D0390915E03BD
:10211000039731F46BEA72E08AE494E00E9487143A
:1021200080915D0390915E03049731F46FEA72E051
:102130008AE494E00E94871482E390E0909357042D
:102140008093560486E590E0909359048093580458
:1021500080EE9FEF90935D0480935C0490935B040A
:1021600080935A0481E080935E0480915B03909198
:102170005C03019731F464EB72E08AE494E00E941E
:10218000871480915B0390915C03029731F468EBB4
:1021900072E08AE494E00E94871480915B0390913E
:1021A0005C03039731F46EEB72E08AE494E00E94E2
:1021B000871480915B0390915C03049731F464EC85
:1021C00072E08AE494E00E94871480915B0390910E
:1021D0005C03059731F46CEC72E08AE494E00E94B1
:1021E000871480915B0390915C03069731F462ED54
:1021F00072E08AE494E00E94871480915B039091DE
:102200005C03449731F467EA72E08AE494E00E9448
:10221000871480915B0390915C03459731F46BEDDB
:1022200072E08AE494E00E94871480915B039091AD
:102230005C03469731F463EE72E08AE494E00E9416
:1022400087146CEE72E08AE494E00E948714809117
:102250005A030E94C01A6EEE72E08AE494E00E9473
:102260008714809159030E94C01A80915A038330C9
:1022700038F080915903833018F088E280932E0360
:102280008FE190E090935D0480935C0490935B04F5
:1022900080935A0481E080935E048EE190E09093F5
:1022A0005704809356048CE690E0909359048093F1
:1022B000580460EF72E08AE494E00E94871480E0A2
:1022C00090E00E94C91A82E891E890935D0480939F
:1022D0005C0490935B0480935A041092570410920C
:1022E000560488E790E0909359048093580462E084
:1022F00073E08AE494E00E948714809149040E946C
:10230000C01A6AE073E08AE494E00E948714809126
:1023100048040E94C01A65E173E08AE494E00E94D8
:102320008714809147040E94C01A68E173E08AE430
:1023300094E00E94871464EC79E080E090E00E94D1
:102340007615DF91CF911F910F910C94590EEF925A
:10235000FF920F931F93CF93DF931F92CDB7DEB7FA
:102360007C01FC0100811181C80169830E943D3616
:102370006981681719F0C8010E944536C7010F909E
:10238000DF91CF911F910F91FF90EF900895CF9221
:10239000DF92EF92FF920F931F93CF93DF936C0125
:1023A0007A018B01C0E0D0E0CE15DF0589F0D801BD
:1023B0006D918D01D601ED91FC910190F081E02DA0
:1023C000C6010995892B11F47E0102C02196ECCF3C
:1023D000C701DF91CF911F910F91FF90EF90DF9098
:1023E000CF900895FC01538D448D252F30E0842F2C
:1023F00090E0821B930B541710F0CF96089501972D
:102400000895FC01918D828D981761F0828DDF0116
:10241000A80FB11D5D968C91928D9F5F9F73928FD7
:1024200090E008958FEF9FEF0895FC01918D828DCC
:10243000981731F0828DE80FF11D858D90E0089599
:102440008FEF9FEF0895FC01918D228D892F90E0F1
:10245000805C9F4F821B91098F739927089588EAAA
:1024600093E00E94231221E0892B09F420E0822FBF
:102470000895FC01848DDF01A80FB11DA35ABF4F41
:102480002C91848D90E001968F739927848FA68973
:10249000B7892C93A089B1898C9180648C93938D9A
:1024A000848D981306C00288F389E02D80818F7D8A
:1024B00080830895EF92FF920F931F93CF93DF9342
:1024C000EC0181E0888F9B8D8C8D981305C0E88985
:1024D000F989808185FD24C0F62E0B8D10E00F5FF9
:1024E0001F4F0F731127E02E8C8DE8120CC00FB612
:1024F00007FCFACFE889F989808185FFF5CFCE0105
:102500000E943912F1CF8B8DFE01E80FF11DE35AC5
:10251000FF4FF0820B8FEA89FB898081806207C0C0
:10252000EE89FF896083E889F989808180648083EE
:1025300081E090E0DF91CF911F910F91FF90EF909C
:102540000895CF93DF93EC01888D8823C9F0EA8941
:10255000FB89808185FD05C0A889B9898C9186FD9C
:102560000FC00FB607FCF5CF808185FFF2CFA88999
:10257000B9898C9185FFEDCFCE010E943912E7CF4A
:10258000DF91CF91089580E090E0892B29F00E949F
:102590002F1281110C9400000895833081F028F4EB
:1025A000813099F08230A1F008958730A9F0883009
:1025B000B9F08430D1F4809180008F7D03C0809188
:1025C00080008F7780938000089584B58F7702C054
:1025D00084B58F7D84BD08958091B0008F7703C04E
:1025E0008091B0008F7D8093B00008953FB7F8943C
:1025F0008091A0039091A103A091A203B091A303A5
:1026000026B5A89B05C02F3F19F00196A11DB11D4D
:102610003FBFBA2FA92F982F8827820F911DA11D88
:10262000B11DBC01CD0142E0660F771F881F991FC5
:102630004A95D1F708952091A6033091A703281752
:10264000390771F49091A4038091A503981741F084
:10265000E091A403F0E0E15AFC4F808190E00895FE
:102660008FEF9FEF089508951F93CF93DF93DC01C1
:102670005C962D913C915D972115310539F481E0EF
:1026800090E013969C938E9312973DC05196ED91D6
:10269000FC91529750969C915097892F80951FB727
:1026A0005E964C915E9741FB772770F941FD6095EE
:1026B000F8944081772311F0492B01C048234083CF
:1026C000E9012197F1F748E0508160FF02C0592BE2
:1026D00001C058235083E9012197F1F766954150D5
:1026E00099F7772321F090818923808303C080812B
:1026F000982B90831FBF5C968D919C915D9701975D
:10270000F1F721E030E0C901DF91CF911F910895E9
:102710002091A6033091A7032817390771F48091FF
:10272000A5032091A40390E0805C9F4F821B910938
:1027300060E470E00E949638089580E090E008958B
:102740002091A6033091A70328173907B9F4909177
:10275000A4038091A503981789F0E091A403F0E009
:10276000E15AFC4F80812091A40330E02F5F3F4F5E
:102770002F7333272093A40390E008958FEF9FEFEA
:102780000895EF92FF920F931F93DC01ED91FC915E
:1027900011971A960D911C911B9718962D913C91AB
:1027A000199700A0F1A1E02D7B0140E050E060E02E
:1027B00070E009951F910F91FF90EF900895FC0133
:1027C000838D882339F06EBD00000DB407FEFDCF68
:1027D0008EB5089528E030E090E8A48DB58D81A5F0
:1027E000492F462319F04C91842B03C04C918095BE
:1027F00084238C93A68DB78D4C9182A5842B8C93CA
:10280000A68DB78D4C9182A5809584238C93969547
:102810002150310911F708950E940539DC01ED912D
:10282000FC910190F081E02D09946115710579F01A
:10283000FB0101900020E9F73197AF01461B570BD0
:10284000DC01ED91FC910280F381E02D099480E0A0
:1028500090E008954F925F926F927F92EF92FF9275
:102860000F931F93CF93DF93CDB7DEB7A1970FB62A
:10287000F894DEBF0FBECDBF7C01FA01CB0119A2D7
:10288000223008F42AE08E010F5D1F4F422E512C9A
:10289000612C712CBF01A30192010E94AA38F90199
:1028A000CA01015011096A3014F4605D01C0695C0D
:1028B000D8016C93232B242B252B61F7B801C7017A
:1028C0000E941514A1960FB6F894DEBF0FBECDBFBF
:1028D000DF91CF911F910F91FF90EF907F906F90BC
:1028E0005F904F9008950F931F93CF93DF93EC0168
:1028F0000E9415148C0161E472E0CE010E9415144F
:10290000800F911FDF91CF911F910F9108950C942B
:1029100015141F920F920FB60F9211242F933F930D
:102920004F935F936F937F938F939F93AF93BF93D7
:10293000EF93FF9388EA93E00E943912FF91EF91A1
:10294000BF91AF919F918F917F916F915F914F91C7
:102950003F912F910F900FBE0F901F9018951F92CF
:102960000F920FB60F9211242F938F939F93EF9393
:10297000FF93E091B803F091B9038081E091BE0329
:10298000F091BF0382FD12C090818091C1038F5FDF
:102990008F732091C203821751F0E091C103F0E0E0
:1029A000E855FC4F958F8093C10301C08081FF9152
:1029B000EF919F918F912F910F900FBE0F901F90CD
:1029C0001895CF93DF93282F30E0F901EA5CFF4E92
:1029D0008491F901EE58FF4ED491F901E25AFF4E6D
:1029E000C491CC2391F081110E94CD12EC2FF0E024
:1029F000EE0FFF1FEC5AFF4EA591B491EC91ED2321
:102A000081E090E021F480E002C080E090E0DF917E
:102A1000CF9108951F93CF93DF93282F30E0F901D2
:102A2000EA5CFF4E8491F901EE58FF4ED491F90112
:102A3000E25AFF4EC491CC23C9F0162F81110E9497
:102A4000CD12EC2FF0E0EE0FFF1FE65BFF4EA591DD
:102A5000B4918FB7F894111105C09C91ED2FE095BA
:102A6000E92302C0EC91ED2BEC938FBFDF91CF9166
:102A70001F910895CF93DF9390E0FC01EE58FF4E35
:102A80002491FC01E25AFF4E8491882361F190E089
:102A9000880F991FFC01E45DFF4EC591D491FC01A4
:102AA000E65BFF4EA591B491611109C09FB7F89400
:102AB0008881209582238883EC912E230BC062307D
:102AC00061F49FB7F8943881822F8095832388839F
:102AD000EC912E2B2C939FBF06C08FB7F894E88102
:102AE0002E2B28838FBFDF91CF9108958F929F92D5
:102AF000AF92BF92CF92DF92EF92FF926B017C0177
:102B00000E94F6124B015C01C114D104E104F104EE
:102B1000F1F00E94F612DC01CB0188199909AA098B
:102B2000BB09883E9340A105B10570F321E0C21AAC
:102B3000D108E108F10888EE880E83E0981EA11CF8
:102B4000B11CC114D104E104F10419F7DDCFFF90E9
:102B5000EF90DF90CF90BF90AF909F908F900895AF
:102B60001F920F920FB60F9211242F933F938F93C2
:102B70009F93AF93BF938091260390912703A091D9
:102B80002803B091290330919F0323E0230F2D37B1
:102B900020F40196A11DB11D05C026E8230F029661
:102BA000A11DB11D20939F038093260390932703BB
:102BB000A0932803B09329038091A0039091A103CF
:102BC000A091A203B091A3030196A11DB11D809312
:102BD000A0039093A103A093A203B093A303BF917A
:102BE000AF919F918F913F912F910F900FBE0F90BA
:102BF0001F9018951F920F920FB60F9211242F93CA
:102C00003F934F935F936F937F938F939F93AF9374
:102C1000BF93EF93FF93E091A603F091A703309742
:102C200009F451C0968DA685B785858591FF04C0AE
:102C30009C91892329F447C09C91892309F043C0C2
:102C4000A389B4899C918589809589238C938689F1
:102C500097890197F1F7608D718DA685B7855585A8
:102C600038E020E0CB010197F1F7822F90E09595B5
:102C70008795282F4C91452309F02068315091F712
:102C8000868D81FD20958091A50390E001968F733C
:102C900099273091A403381749F0A091A503B0E01B
:102CA000A15ABC4F2C938093A50303C0868D8160ED
:102CB000868F828D938D0197F1F7A389B4899C91BA
:102CC0008589892B8C93FF91EF91BF91AF919F9153
:102CD0008F917F916F915F914F913F912F910F90C5
:102CE0000FBE0F901F901895E091A603F091A703D7
:102CF000E817F90769F4A389B4899C9185898095BF
:102D000089238C931092A7031092A60381E0089563
:102D100080E008950F931F93CF93DF931F92CDB759
:102D2000DEB78C01809145049091460469830E942E
:102D30001E0ED8019296ED91FC91939790819C96EE
:102D40008C919C97892B80839096ED91FC91919723
:102D500090819B968C918095892380836981C8019D
:102D60000E94DF13D8019096ED91FC91919790818C
:102D70009B968C91892B80830F90DF91CF911F912F
:102D80000F910C941D0E0F931F93CF93DF931F92FF
:102D9000CDB7DEB78C0180914504909146046983DC
:102DA0000E941E0ED8019296ED91FC91939790810E
:102DB0009C968C919C978095892380839096ED9129
:102DC000FC91919790819B968C918095892380832B
:102DD0006981C8010E94DF13D8019096ED91FC91A2
:102DE000919790819B968C91892B80830F90DF9196
:102DF000CF911F910F910C941D0E611102C060E2E2
:102E000001C061E20C94C3161F93CF93DF93EC01D2
:102E1000162F66E30E94C316612F63706D8B8A8D37
:102E2000623089F16330A9F16130D1F0823011F460
:102E300060EC01C068ECCE010E948A1680E890E048
:102E4000998788878A8D813019F480E890E002C0E4
:102E500080EA90E09B878A87DF91CF911F91089548
:102E6000823011F460EA01C068EACE010E948A163D
:102E70008A8D813019F480E890E002C080EA90E009
:102E800099878887E2CF823011F460E0D4CF68E080
:102E9000D2CF823011F460E6E8CF68E6E6CFEF9259
:102EA000FF920F931F93CF93DF9300D0CDB7DEB780
:102EB0007C01162F6AE229834A830E94C31660E0D0
:102EC000C7010E948A16F70185A5612F680FC70107
:102ED0000E948A1660E0C7010E948A16F70185A544
:102EE0002981622F680FC7010E948A166BE2C70111
:102EF0000E94C31660E0C7010E948A16F70186A5EA
:102F00004A81642F680FC7010E948A1660E0C701DA
:102F10000E948A16F70186A5602F680FC7010E94DC
:102F20008A166CE2C7010F900F90DF91CF911F912D
:102F30000F91FF90EF900C94C316AF92BF92CF9277
:102F4000DF92EF92FF920F931F93CF93DF93EC01E9
:102F50005901680128853985621773070CF05CC038
:102F60008A859B85481759070CF056C0FB01EA0D6E
:102F7000FB1D2E173F071CF45901A61AB70A9A0128
:102F80002C0D3D1D821793071CF46C01C41AD50A41
:102F90000FEF040F0C0D2FEF260F2A0DCE010E940C
:102FA0004F1780914504909146040E941E0EEAA19D
:102FB000FBA190818CA5892B8083E8A1F9A1908148
:102FC0008BA58095892380831C141D049CF48501A6
:102FD000101611065CF46F2DCE010E94DF136E2DCA
:102FE000CE010E94DF1301501109F2CF81E0C81A0F
:102FF000D108EACFE8A1F9A190818BA5892B808324
:10300000DF91CF911F910F91FF90EF90DF90CF90C4
:10301000BF90AF900C941D0EDF91CF911F910F9137
:10302000FF90EF90DF90CF90BF90AF900895DF9228
:10303000EF92FF920F931F93CF93DF93EC017901EF
:10304000D02E88859985681779070CF047C02A85A6
:103050003B85421753070CF041C09B012E0D3F1DCD
:10306000821793071CF47C01E61AF70A2FEF260F4C
:103070002E0D042FCE010E944F1780914504909190
:1030800046040E941E0EEAA1FBA190818CA5892B0B
:103090008083E8A1F9A190818BA580958923808305
:1030A000E114F10461F0612FCE010E94DF136D2D58
:1030B000CE010E94DF1381E0E81AF108F1CFE8A108
:1030C000F9A190818BA5892B8083DF91CF911F91EE
:1030D0000F91FF90EF90DF900C941D0EDF91CF9138
:1030E0001F910F91FF90EF90DF900895DF92EF9284
:1030F000FF920F931F93CF93DF93EC017901D02EB2
:1031000088859985681779070CF047C08A859B8563
:10311000481759070CF041C09A012E0D3F1D821728
:1031200093071CF47C01E41AF50A0FEF040F0E0D4F
:10313000262FCE010E944F1780914504909146049E
:103140000E941E0EEAA1FBA190818CA5892B808391
:10315000E8A1F9A190818BA5809589238083E11452
:10316000F10461F0612FCE010E94DF136D2DCE01BD
:103170000E94DF1381E0E81AF108F1CFE8A1F9A17C
:1031800090818BA5892B8083DF91CF911F910F9127
:10319000FF90EF90DF900C941D0EDF91CF911F9167
:1031A0000F91FF90EF90DF900895EF92FF920F93B1
:1031B0001F93CF93DF931F92CDB7DEB77C01CB0176
:1031C000122F77FD53C0D70118966D917C911997F6
:1031D000861797070CF04AC057FD48C01A966D91A4
:1031E0007C911B97461757070CF040C001E0040F75
:1031F00021E0280F682FC70139830E944F17809163
:103200004504909146040E941E0ED7019296ED91BE
:10321000FC91939790819C968C919C97892B8083AD
:103220009096ED91FC91919790819B968C918095D1
:10323000892380833981632FC7010E94DF13612FA7
:10324000C7010E94DF13D7019096ED91FC919197F1
:1032500090819B968C91892B80830F90DF91CF91E9
:103260001F910F91FF90EF900C941D0E0F90DF9126
:10327000CF911F910F91FF90EF9008952F923F9261
:103280004F925F926F927F928F929F92AF92BF9276
:10329000CF92DF92EF92FF920F931F93CF93DF9322
:1032A0006C015B01EA0181E090E04C01841A950A0F
:1032B00066247724641A750A660C771CE12CF12CBD
:1032C000822F8470582E822F8270482E822F887011
:1032D000382E2170222EEC16FD060CF073C097FCE0
:1032E00006C0219782E0680E711C860C971C8FEF38
:1032F000E81AF80AC701880F991F0196880E991ECF
:103300005520B1F09801A5014C0F5D1FB7016C0D60
:103310007D1D8AE494E00E94670D9801A7014A0D83
:103320005B1DB6016C0F7D1F8AE494E00E94670D5F
:103330004420B1F09801A5014C1B5D0BB7016C0D49
:103340007D1D8AE494E00E94670D9801A5014E1945
:103350005F09B6016C0F7D1F8AE494E00E94670D3F
:103360003320B1F09801A7014A0D5B1DB6016C1B1B
:103370007D0B8AE494E00E94670D9801A5014C0F33
:103380005D1FB6016E197F098AE494E00E94670D03
:10339000222009F4A0CF9801A5014E195F09B601BA
:1033A0006C1B7D0B8AE494E00E94670D9801A501D7
:1033B0004C1B5D0BB6016E197F098AE494E00E94F4
:1033C000670D89CFDF91CF911F910F91FF90EF9003
:1033D000DF90CF90BF90AF909F908F907F906F9035
:1033E0005F904F903F902F900895CF92DF92EF9291
:1033F000FF920F931F93CF93DF9377FF1DC06A0156
:103400007B01EC016DE20E940E148C0144275527CC
:10341000BA014C195D096E097F092AE0CE010E94AC
:103420002A14800F911FDF91CF911F910F91FF9070
:10343000EF90DF90CF9008952AE0DF91CF911F9118
:103440000F91FF90EF90DF90CF900C942A14109280
:10345000940410929304109292041092910410928A
:10346000900410928F048DEC90E0909396048093DA
:10347000950490918504963108F057C025E530E019
:103480003093900420938F042BEC30E0309392041F
:103490002093910420E930E0309394042093930426
:1034A00020916800983050F031E09E3008F430E010
:1034B00081E001C0880F3A95EAF701C084E0822BD1
:1034C00080936800983038F09E3040F0963148F094
:1034D00020E030E008C02DE630E005C02BE630E00B
:1034E00002C02CE630E030938D0420938C04983099
:1034F00030F481E001C0880F9A95EAF70EC0292FB9
:1035000030E09E3018F42850310902C02E503109A5
:1035100081E001C0880F2A95EAF780938E0480919C
:103520009504909196040197F1F7809193049091FE
:103530009404892B21F18091A6039091A70324E0A4
:1035400089379207E1F0009711F00E94741680917C
:1035500097048E7F809397041092A5031092A40382
:1035600089E794E09093A7038093A603E0918C04ED
:10357000F0918D04908180918E04892B8083089531
:10358000482F50E060E070E02AE08AE494E00C9478
:103590002A142091620430916304009749F0232B90
:1035A00099F420915804309159042A5F3F4F08C084
:1035B000232B51F0209158043091590426503109A1
:1035C00030935904209358049093630480936204C9
:1035D0000895CF93DF93EC0161E085E00E943A15F6
:1035E000209711F460E004C0CF3FD10531F461E0D1
:1035F00085E0DF91CF910C940A15EBE3F0E1E491C3
:10360000E330F9F048F4E130B9F0E230A1F584B5E7
:10361000806284BDC8BD34C0E730E9F0E83019F1FC
:10362000E43049F580918000806280938000D093DF
:103630008B00C0938A0024C084B5806884BDC7BD58
:103640001FC080918000806880938000D0938900A3
:10365000C093880015C08091B00080688093B0004E
:10366000C093B3000DC08091B00080628093B00021
:10367000C093B40005C0C038D1050CF0B8CFB2CFAC
:10368000DF91CF910895CF92DF92EF92FF920F9347
:103690001F93CF93DF93EC012196FC01149111232A
:1036A00009F437C0FE0164918AE494E00E94C316D5
:1036B0006E01F2E0CF0ED11CFE013196C4910C2FA9
:1036C0000078CF777601DC2FD15050F0F70164916C
:1036D0008AE494E00E948A16FFEFEF1AFF0AF4CF03
:1036E000C6018C0F911DEC01002389F07C019FEF36
:1036F000E91AF90AFE01649170E06F3F710511F457
:1037000064EF71E080E090E00E947615E7011150CF
:10371000C6CFDF91CF911F910F91FF90EF90DF9077
:10372000CF9008952F923F924F925F926F927F9227
:103730008F929F92AF92BF92CF92DF92EF92FF92C1
:103740000F931F93CF93DF9300D000D000D0CDB75D
:10375000DEB72C013B015C834B8319011E830D8373
:103760005801B194A194B108AA0CBB1C4A018A0C5F
:103770009B1C6801C40CD51C87019401AB01B601E8
:103780008AE494E00E944F0DC301820D931D9A8339
:103790008983AC01415051099401B6018AE494E057
:1037A0000E944F0DA20CB31CED81FE816E0E7F1E98
:1037B0009501A301B2018AE494E00E945B0D8B8124
:1037C0009C81480E591EB201615071099501A301F7
:1037D0008AE494E00E945B0D21E04D815E81B3019B
:1037E000C6010E943E19ED81FE814E1A5F0AF1E08A
:1037F0004F1A510822E04D815E81B301C2010E943F
:103800003E19A980BA808D819E81A81AB90A91E0DB
:10381000A91AB10824E04D815E81B501C2010E9460
:103820003E1928E04D815E81B501C6010E943E1916
:1038300026960FB6F894DEBF0FBECDBFDF91CF91B5
:103840001F910F91FF90EF90DF90CF90BF90AF90BE
:103850009F908F907F906F905F904F903F902F90B0
:1038600008954F925F926F927F928F929F92AF9244
:10387000BF92CF92DF92EF92FF920F931F93CF935D
:10388000DF936C015B014A0139012801E7018FE1F7
:10389000E82EF12C89019A01AB01B6018AE494E08B
:1038A0000E94D00B8E019201A301B4018AE494E03E
:1038B0000E94D00B85019601AE01B2018AE494E02A
:1038C0000E94D00BDF91CF911F910F91FF90EF904D
:1038D000DF90CF90BF90AF909F908F907F906F9030
:1038E0005F904F9008950F931F93CF93DF93EC0158
:1038F000462F50E060E070E02AE00E942A148C011C
:1039000061E472E0CE010E941514800F911FDF91D7
:10391000CF911F910F910895CF93DF93CDB7DEB76D
:103920002A970FB6F894DEBF0FBECDBF789484B54A
:10393000826084BD84B5816084BD85B5826085BDAB
:1039400085B5816085BD80916E00816080936E0039
:10395000109281008091810082608093810080912B
:1039600081008160809381008091800081608093DC
:1039700080008091B10084608093B1008091B0009C
:1039800081608093B00080917A00846080937A0097
:1039900080917A00826080937A0080917A008160C1
:1039A00080937A0080917A00806880937A001092E8
:1039B000C10060E084E00E943A1560E087E00E9468
:1039C0003A1560E086E00E943A1561E085E00E94C9
:1039D0003A15E091B803F091B90382E08083E09159
:1039E000B403F091B5031082E091B603F091B703F0
:1039F00087E680831092C003E091BC03F091BD0381
:103A000086E08083E091BA03F091BB0380818061FE
:103A10008083E091BA03F091BB038081886080834A
:103A2000E091BA03F091BB03808180688083E091CC
:103A3000BA03F091BB0380818F7D808364E170E0E5
:103A400080E090E00E9476156EE571E088EA93E0F0
:103A50000E9473140E94271A64E170E080E090E0F5
:103A60000E94761565E571E088EA93E00E94731480
:103A700064E170E080E090E00E9476150E945F0EA5
:103A80000E94210E22242394312C30EEA32E37E005
:103A9000B32E84E00E94E114082F8093570386E040
:103AA0000E94E114182F8093560387E00E94E114CE
:103AB00080935503013009F059C0113009F056C008
:103AC00061E771E088EA93E00E9487140E94590E32
:103AD0008DE090E0909357048093560480E290E04C
:103AE000909359048093580410935E0480E098EFFB
:103AF00090935D0480935C0490935B0480935A04DC
:103B000065E871E08AE494E00E94871460914904BA
:103B10001A821982CE0101960E94A7116091480471
:103B20003A822982CE0101960E94A7116091470432
:103B300082E090E09A838983CE0101960E94A711CA
:103B400068EB7BE080E090E00E94761565E971E02B
:103B50008AE494E00E94871468EE73E080E090E0CD
:103B60000E9476150E94590E10930401809157030C
:103B700081111FC0809156038130D9F48091470490
:103B80008F5F833019F08093470402C0109247047E
:103B90000E94590E66E970E080E090E00E94761580
:103BA00081E08093040166E970E080E090E00E948B
:103BB000761580915703813009F043C080915503F9
:103BC00081113FC0809149048A508B3008F483ED05
:103BD000809349046EE971E088EA93E00E948714BB
:103BE0006091490488EA93E00E94731C8091490423
:103BF00090E00E94E91A20914904269530E090EE69
:103C0000E92EFF24FA940FE710E04FE750E060E060
:103C100070E08AE494E00E94D00B62E370E080E000
:103C200090E00E94761520914904269530E0E12C21
:103C3000F12C4FE750E060E070E08AE494E00E94ED
:103C4000D00B80915703813009F041C0809155031A
:103C50008130E9F5809148048A5009F487E980931E
:103C6000480460EB71E088EA93E00E948714609159
:103C7000480488EA93E00E94731C8091480490E015
:103C80000E94E91A20914804269530E08FE1E82E41
:103C9000F12C0FE710E04FE750E060E070E08AE4BD
:103CA00094E00E94D00B62E370E080E090E00E941C
:103CB000761520914804269530E0E12CF12C4FE751
:103CC00050E060E070E08AE494E00E94D00B8091C4
:103CD0005503811103C08091490404C0813029F447
:103CE0008091480490E00E94E91A5090040191E00C
:103CF0005912FEC4109254031092530310925203AF
:103D0000109251031092500310924F0310924E03E1
:103D100010924A0310924B0310924C0310924D03E1
:103D200010924903109248031092470310924603E1
:103D30001092450310923B0310923C0310923D03F6
:103D400010923E0310923F031092410310924303DE
:103D50001092440310923A031092310310924203DE
:103D600010924003109237031092360310923503DD
:103D700010923403109239031092380310923303D7
:103D8000109232033092030120920201309201011D
:103D9000209200018091470481508E3F08F4CDC2EB
:103DA00084E190E0909357048093560490935904D3
:103DB0008093580450925E049FE1C92ED12CD0927A
:103DC0005D04C0925C04D0925B04C0925A0464EC1F
:103DD00071E08AE494E00E94731468EC70E080E083
:103DE00090E00E9476150E94590EB0925D04A09258
:103DF0005C04B0925B04A0925A0482E090E090933D
:103E00005704809356049093590480935804509219
:103E10005E046DEC71E08AE494E00E94731421E288
:103E2000622E712C709257046092560482E090E0EA
:103E3000909359048093580450925E0461ED71E0B0
:103E40008AE494E00E9473143FE1E32EF12C0CE02D
:103E500010E02FE930E040E050E060E070E08AE4FC
:103E600094E00E94710B28E230E040E050E06EE107
:103E700070E08AE494E00E94710B82E090E09093FD
:103E800057048093560441E1842E912C909259045A
:103E90008092580450925E04B0925D04A0925C043B
:103EA000B0925B04A0925A0467ED71E08AE494E05A
:103EB0000E947314709257046092560490925904B1
:103EC0008092580450925E046BED71E08AE494E0B5
:103ED0000E9473142FE930E04FE050E060E070E0A2
:103EE0008AE494E00E94710B28E230E04FE050E059
:103EF0006EE170E08AE494E00E94710B2EE130E004
:103F00004FE050E06AE570E08AE494E00E94710BB3
:103F10008CE590E090935704809356049092590456
:103F20008092580450925E04B0925D04A0925C04AA
:103F3000B0925B04A0925A0462EE71E08AE494E0CD
:103F40000E94731485E790E0909357048093560481
:103F5000909259048092580450925E0466EE71E08B
:103F60008AE494E00E94731482E090E090935704F6
:103F70008093560480E290E0909359048093580413
:103F800050925E04B0925D04A0925C04B0925B0417
:103F9000A0925A046DEE71E08AE494E00E947314DA
:103FA000709257046092560480E290E09093590416
:103FB0008093580450925E04809144030E94C01A7A
:103FC00061EF71E08AE494E00E9473142FE930E01D
:103FD0004EE150E060E070E08AE494E00E94710BF2
:103FE00028E230E04EE150E06EE170E08AE494E0D7
:103FF0000E94710B88E190E09093570480935604DF
:1040000050E3652E712C70925904609258045092BE
:104010005E04B0925D04A0925C04B0925B04A09236
:104020005A0464EF71E08AE494E00E94731486E11C
:1040300090E090935704809356040CE310E01093A3
:1040400059040093580484E080935E0460EE862E49
:1040500099249A9490925D0480925C0490925B04FF
:1040600080925A046AE072E08AE494E00E94731439
:104070008CE690E090935704809356047092590414
:104080006092580450925E04B0925D04A0925C0469
:10409000B0925B04A0925A0468EF71E08AE494E065
:1040A0000E94731483E790E0909357048093560422
:1040B000109359040093580485E080935E04909215
:1040C0005D0480925C0490925B0480925A046AE0E2
:1040D00072E08AE494E00E94731472E4E72EF12CFB
:1040E0000FE510E022E430E041E450E063E370E0EB
:1040F00080E590E00E94311CE6E4EE2EF12C26E4EF
:1041000030E041E450E065E570E080E590E00E9439
:10411000311C90925D0480925C0490925B048092CA
:104120005A0488E290E09093570480935604FDE689
:104130006F2E712C709259046092580412E0109303
:104140005E046AE072E08AE494E00E947314909244
:104150005D0480925C0490925B0480925A0484E037
:1041600090E09093570480935604709259046092A3
:10417000580410935E046AE072E08AE494E00E94BE
:104180007314B0925D04A0925C04B0925B04A092A0
:104190005A0484E290E09093570480935604A2E678
:1041A0006A2E712C709259046092580450925E04E9
:1041B00060E072E08AE494E00E9473143092570445
:1041C00020925604709259046092580450925E04F2
:1041D00064E072E08AE494E00E94731490925D04BB
:1041E00080925C0490925B0480925A0484E690E092
:1041F0009093570480935604BEE68B2E912C909298
:1042000059048092580410935E0468E072E08AE4D6
:1042100094E00E947314D0925D04C0925C04D0922A
:104220005B04C0925A048BE890E09093570480930B
:104230005604909259048092580450925E046CE0A7
:1042400072E08AE494E00E94731485E990E0909310
:1042500057048093560412E7C12ED12CD0925904F2
:10426000C092580450925E046FE072E08AE494E0D9
:104270000E94731488E990E0909357048093560449
:1042800086E790E0909359048093580450925E041E
:1042900063E372E08AE494E00E94731484E490E0A3
:1042A00090935704809356048EE590E090935904C0
:1042B0008093580450925E04B0925D04A0925C0416
:1042C000B0925B04A0925A0461E172E08AE494E047
:1042D0000E9473140FE1E02EF12C07E010E020E1C2
:1042E00030E048E250E06AE570E08CE390E00E9444
:1042F000921B8FE390E09093570480935604D092E2
:104300005904C092580450925E04B0925D04A09289
:104310005C04B0925B04A0925A0466E172E08AE405
:1043200094E00E94731420E130E048E250E06EE631
:1043300070E08CE390E00E94921BD090470491E0E3
:10434000D912A3C184E190E090935704809356045E
:104350009093590480935804D0925E040FE110E0CA
:1043600010935D0400935C0410935B0400935A0463
:104370006DE172E08AE494E00E94731464EF71E0EE
:1043800080E090E00E9476150E94590ED0925E0463
:1043900010935D0400935C0410935B0400935A0433
:1043A0008BE090E090935704809356043092590428
:1043B0002092580464E272E08AE494E00E94871438
:1043C00010935704009356043092590420925804D5
:1043D0006CE372E08AE494E00E94871483E390E047
:1043E00090935704809356043092590420925804B5
:1043F00066E272E08AE494E00E94871487E490E029
:104400009093570480935604309259042092580494
:1044100068E272E08AE494E00E9487148BE590E001
:104420009093570480935604309259042092580474
:1044300060E073E08AE494E00E9487148FE690E0E5
:104440009093570480935604309259042092580454
:104450006AE272E08AE494E00E94871483E890E0C4
:104460009093570480935604309259042092580434
:104470006CE272E08AE494E00E94871487E990E09D
:104480009093570480935604309259042092580414
:104490006EE272E08AE494E00E94871404EEE02E5B
:1044A00008EAF02E03E010E024E130E048E050E0BC
:1044B0006AE070E080E090E00E94921B24E130E02E
:1044C00048E050E06AE070E08AE090E00E94921BD1
:1044D00024E130E048E050E06AE070E084E190E000
:1044E0000E94921B24E130E048E050E06AE070E076
:1044F0008EE190E00E94921B24E130E048E050E021
:104500006AE070E088E290E00E94921B24E130E0D3
:1045100048E050E06AE070E082E390E00E94921B85
:1045200024E130E048E050E06AE070E08CE390E0A5
:104530000E94921B24E130E048E050E06AE070E025
:1045400086E490E00E94921B24E130E048E050E0D5
:104550006AE070E080E590E00E94921B24E130E088
:1045600048E050E06AE070E08AE590E00E94921B2B
:1045700024E130E048E050E06AE070E084E690E05A
:104580000E94921B24E130E048E050E06AE070E0D5
:104590008EE690E00E94921B24E130E048E050E07B
:1045A0006AE070E088E790E00E94921B24E130E02E
:1045B00048E050E06AE070E082E890E00E94921BE0
:1045C00024E130E048E050E06AE070E08CE890E000
:1045D0000E94921B24E130E048E050E06AE070E085
:1045E00086E990E00E94921B80EEE82EFF24FA9468
:1045F00009E110E022E230E043E650E063E570E0DC
:104600008AE494E00E94710B03E010E024E030E0C3
:1046100041E650E066E570E08AE494E00E94710BA8
:1046200024E030E041E650E06EE670E08AE494E099
:104630000E94710B8DE290E0909357048093560492
:1046400083E690E09093590480935804D0925E04DE
:104650008FEF97E090935D0480935C0490935B04EC
:1046600080935A0460E372E08AE494E00E94731439
:1046700082E08093330380933203809348038093D6
:10468000470380934603809345038091470482301B
:1046900069F584E190E090935704809356049093D9
:1046A00059048093580481E080935E048FE190E088
:1046B00090935D0480935C0490935B0480935A0410
:1046C00065E372E08AE494E00E94731464EF71E0A1
:1046D00080E090E00E9476150E94590EB0925D0431
:1046E000A0925C04B0925B04A0925A041092040160
:1046F0008091570381110C94B7308091560381113A
:104700000C94B73089E794E00E94881397FF02C0A9
:104710000C94B73089E794E00E94A0136C0162E02A
:1047200070E080E090E00E947615C114D10421F081
:10473000D7FE02C00C94B73080912F0390913003C4
:104740008F30910514F00C94B7300196909330039C
:1047500080932F036EE372E088EA93E00E9487144F
:1047600026010D2C000C66087708B301A20188EA27
:1047700093E00E94F51962E070E080E090E00E9412
:10478000761580912F0390913003019709F021C293
:104790008091540390E08C159D0509F41AC294E5AC
:1047A0009C1518F0C092440303C085E58093440330
:1047B0008091470481115CC0E12CF12C0AE010E0EB
:1047C0002DE030E04FE150E06FE170E08AE494E0EA
:1047D0000E949D1790904403692D70E026E530E01B
:1047E000261B370B6A5B7F4F4FE150E08AE494E071
:1047F0000E949D1789E0891510F00C94DA3081E24F
:1048000090E0909357048093560480E290E0909358
:1048100059048093580481E080935E04B0925D0453
:10482000A0925C04B0925B04A0925A0494E6999E14
:10483000A0011124052E000C660B770B8AE494E08E
:104840000E94F51961E472E08AE494E00E94151474
:104850002091440330E0E12C18EFF12E08E010E045
:104860004FE150E067E470E08AE494E00E949D1715
:1048700080914704813009F0ACC1E12CF12C04E2B5
:1048800010E024E330E042E250E067E370E08AE4C5
:1048900094E00E949D17109144031A3010F40C9478
:1048A000DE3085E390E090935704809356048EE3C6
:1048B00090E0909359048093580482E080935E04C2
:1048C00082EB9AE00E94C91AB0925D04A0925C0447
:1048D000B0925B04A0925A0484E6189FA0011124B0
:1048E000052E000C660B770B8AE494E00E94F51904
:1048F00080E090E00E94C91A80914403853028F03E
:10490000B0EEEB2EB7E0FB2E02C0E12CF12C02E062
:1049100010E021E130E044E050E06CE070E082E043
:1049200090E00E942333809144038A3028F0A0EE67
:10493000EA2EA7E0FA2E02C0E12CF12C02E010E0F2
:1049400021E130E044E050E06CE070E08CE090E089
:104950000E942333809144038F3028F0F0EEEF2E35
:10496000F7E0FF2E02C0E12CF12C02E010E021E183
:1049700030E044E050E06CE070E086E190E00E94BE
:10498000233380914403843128F0E0EEEE2EE7E0FB
:10499000FE2E02C0E12CF12C02E010E021E130E01B
:1049A00044E050E06CE070E080E290E00E9423334D
:1049B00080914403893128F070EEE72E77E0F72EDE
:1049C00002C0E12CF12C02E010E021E130E044E0F3
:1049D00050E06CE070E08AE290E00E942333809126
:1049E00044038E3128F060EEE62EFF24FA9402C0D4
:1049F000E12CF12C02E010E021E130E044E050E055
:104A00006CE070E084E390E00E94233380914403E3
:104A1000833228F050EEE52EFF24FA9402C0E12CF8
:104A2000F12C02E010E021E130E044E050E06CE0E5
:104A300070E08EE390E00E9423338091440388323B
:104A400028F040EEE42EFF24FA9402C0E12CF12C71
:104A500002E010E021E130E044E050E06CE070E082
:104A600088E490E00E942333809144038D3228F043
:104A700030EAE32E3DEFF32E02C0E12CF12C02E0F0
:104A800010E021E130E044E050E06CE070E082E5CD
:104A900090E00E94233380914403823328F020EA7F
:104AA000E22E2DEFF22E02C0E12CF12C02E010E0FC
:104AB00021E130E044E050E06CE070E08CE590E013
:104AC0000E94233380914403873328F090EAE92E33
:104AD0009DEFF92E02C0E12CF12C02E010E021E163
:104AE00030E044E050E06CE070E086E690E00E9448
:104AF0002333809144038C3320F0E12C88EFF82E8F
:104B000002C0E12CF12C02E010E021E130E044E0B1
:104B100050E06CE070E080E790E00E9423338091E9
:104B20004403813420F0E12C08EFF02E02C0E12C88
:104B3000F12C02E010E021E130E044E050E06CE0D4
:104B400070E08AE790E00E9423338091440386342A
:104B500020F0E12C18EFF12E02C0E12CF12C02E044
:104B600010E021E130E044E050E06CE070E084E8E7
:104B700090E00E942333809144038B3428F0B6EBFD
:104B8000EB2EBBE8FB2E02C0E12CF12C02E010E082
:104B900021E130E044E050E06CE070E08EE890E02D
:104BA0000E94233380914403803528F0A6EBEA2E3F
:104BB000ABE8FA2E02C0E12CF12C02E010E021E17A
:104BC00030E044E050E06CE070E088E990E00E9462
:104BD000233380912F0390913003029709F08DC009
:104BE0008091530390E08C159D0509F486C0C09216
:104BF000430380914704811132C0E12CF12C0FE076
:104C000010E022E230E04EE650E064E670E08AE434
:104C100094E00E949D1780EE9FEF90935D04809337
:104C20005C0490935B0480935A0493E69C1518F0FF
:104C30008FE690E002C084E690E090935704809362
:104C400056048EE690E0909359048093580482E0D5
:104C500080935E046C2D8AE494E00E94731C809122
:104C60004704813009F049C0FFE1EF2EF12C02E04A
:104C700010E02CE130E046E250E061E670E088E2CE
:104C800090E00E94921B8FEF97E090935D048093D9
:104C90005C0490935B0480935A04E12CF12C0FE0A8
:104CA00010E022E230E04DE650E06AE270E08AE493
:104CB00094E00E949D1780EE9FEF90935D04809397
:104CC0005C0490935B0480935A0480914303843680
:104CD00018F421E330E002C02AE230E030935704B8
:104CE000209356042DE630E0309359042093580465
:104CF00092E090935E040E94C01A80912F039091DD
:104D00003003039709F092C08091520390E08C1514
:104D10009D0509F48BC094E69C1518F0C0924203DF
:104D200003C084E6809342038091470481117EC0D2
:104D300080EE9FEF90935D0480935C0490935B04FE
:104D400080935A04E12CF12C0AE010E024E130E0D9
:104D500041E050E06FE170E08AE494E00E949D172A
:104D600090904203692D70E080E090E00E946F37E0
:104D70002DE33AE047E55FE30E9424386B837C83B0
:104D80008D839E839B01AC0160E070E08CEA92E42D
:104D90000E9453360E9437376F83788789879A87B6
:104DA00020E030E04CE852E46B817C818D819E8173
:104DB0000E9454360E9437372F81388541E050E0F9
:104DC0008AE494E00E949D1781E290E0909357045A
:104DD0008093560482E090E09093590480935804A5
:104DE00081E080935E04692D8AE494E00E94731C44
:104DF0006091420370E080E090E00E946F372DE305
:104E00003AE047E55FE30E9424380E943737EE24FA
:104E1000EA94E7E0FE2E08E010E09B0142E050E05B
:104E200067E470E08AE494E00E949D1780912F036C
:104E300090913003049709F027C1C114D10409F4FB
:104E400023C18091020190910301C816D90609F48B
:104E50001BC1D0920101C0920001809147048111D1
:104E600034C0E12CF12C09E010E024E130E041E114
:104E700050E06BE770E08AE494E00E949D1780EEBA
:104E80009FEF90935D0480935C0490935B04809308
:104E90005A048BE790E0909357048093560481E185
:104EA00090E0909359048093580481E080935E04CD
:104EB00080912E03A601481B5109052E000C660B9C
:104EC000770B8AE494E00E94F519909147049B8344
:104ED000913009F06AC05FE1E52EF12C02E010E0AC
:104EE0002CE130E046E250E061E670E080E090E0E6
:104EF0000E94921B88248A9467E0962E90925D040B
:104F000080925C0490925B0480925A043092570421
:104F10002092560483E690E09093590480935804BD
:104F20008B8180935E0464E472E08AE494E00E94E2
:104F30008714E12CF12C00E110E023E230E04BE695
:104F400050E061E070E08AE494E00E949D17409197
:104F50000001509101014436510514F40C94E230E3
:104F600082E090E090935704809356048DE690E0A1
:104F7000909359048093580480E098EF90935D04D7
:104F800080935C0490935B0480935A0482E0809346
:104F90005E0480912E03481B5109052E000C660B00
:104FA000770B8AE494E00E94F519809147048230DF
:104FB00009F06AC03FE1E32EF12C02E010E02CE1A1
:104FC00030E046E250E062E070E080E090E00E9475
:104FD000921B88248A9447E0942E90925D048092DC
:104FE0005C0490925B0480925A04309257042092A1
:104FF000560484E090E0909359048093580481E033
:1050000080935E0464E472E08AE494E00E94871472
:10501000E12CF12C00E110E023E230E04CE050E024
:1050200061E070E08AE494E00E949D1740910001E5
:10503000509101014436510514F40C94F83082E08B
:1050400090E090935704809356048EE090E0909304
:1050500059048093580480E098EF90935D04809306
:105060005C0490935B0480935A0482E080935E0416
:1050700080912E03481B5109052E000C660B770BFF
:105080008AE494E00E94F51980912F0390913003F7
:10509000059709F08DC08091510390E08C159D0516
:1050A00009F486C0C092410380914704811127C052
:1050B000E12CF12C0FE010E02CE030E04DE650E068
:1050C00064E070E08AE494E00E949D1780EE9FEF18
:1050D00090935D0480935C0490935B0480935A04E6
:1050E00084E090E090935704809356048DE690E01E
:1050F000909359048093580482E080935E048091D9
:105100004704813039F5E12CF12C00E110E020E179
:1051100030E04EE650E063E970E08AE494E00E94FB
:105120009D178FEF97E090935D0480935C049093BC
:105130005B0480935A0483E990E090935704809332
:1051400056048EE690E0909359048093580482E0D0
:1051500080935E0480914704823039F5E12CF12C74
:1051600009E110E022E130E044E650E066E870E05A
:105170008AE494E00E949D1780EE9FEF90935D0477
:1051800080935C0490935B0480935A0486E890E0DB
:10519000909357048093560484E690E090935904CA
:1051A0008093580483E080935E048C2D0E94C01A83
:1051B00080912F03909130030697C1F580915003A1
:1051C00090E08C159D0591F1C092400380914704B9
:1051D00081112CC0E12CF12C0FE010E02CE030E02C
:1051E0004DE650E068E270E08AE494E00E949D178A
:1051F0008FEF97E090935D0480935C0490935B0441
:1052000080935A0488E290E0909357048093560468
:105210008DE690E0909359048093580482E0809347
:105220005E046C2D8AE494E00E94731C80912F032D
:10523000909130030B9709F023C1C301B2010E9482
:105240006F372B013C019B01AC0160914A037091C7
:105250004B0380914C0390914D030E94C0368823EC
:1052600009F40EC140923C0350923D0360923E030C
:1052700070923F0380914704811138C080EE9FEF08
:1052800090935D0480935C0490935B0480935A0434
:10529000E12CF12C0AE010E02AE130E040E150E09E
:1052A0006FE170E08AE494E00E949D1780E290E054
:1052B000909357048093560481E190E090935904B1
:1052C0008093580481E080935E0420E030E040E267
:1052D00051E4C301B2010E94C53642E00E945F352D
:1052E00061E472E08AE494E00E941514809147041E
:1052F000813009F0C5C025E530E030935704209394
:1053000056042CE630E030935904209358048093DF
:105310005E0440903C0350903D0360903E037090CB
:105320003F0320E030E04AEF52E4C301B2010E94A3
:105330001F381816BCF42FE1E22EF12C05E110E025
:105340002FE130E045E650E064E570E08AE494E067
:105350000E949D17B0925D04A0925C04B0925B0421
:10536000A0925A0420E030E044EE52E4C301B201BE
:105370000E941F38181624F520E030E04CEF52E46C
:10538000C301B2010E94C03687FF1AC092E8E92E1D
:1053900091E8F92E05E110E02FE130E045E650E01C
:1053A00065E570E08AE494E00E949D1780EA9DEF35
:1053B00090935D0480935C0490935B0480935A0403
:1053C00020E030E046EE52E4C301B2010E94C03654
:1053D00087FF35C0E12C88EFF82E05E110E02FE1C2
:1053E00030E045E650E065E570E08AE494E00E9434
:1053F0009D1787E590E0909357048093560486E6C6
:1054000090E090935904809358046BE472E08AE42E
:1054100094E00E94871410925D0410925C04109234
:105420005B0410925A0485E590E0909357048093B2
:10543000560480E790E0909359048093580420919B
:105440004A0330914B0340914C0350914D036091BE
:105450003C0370913D0380913E0390913F030E9475
:10546000543620E030E040E251E40E94C53620E0AE
:1054700030E040E05FE30E94243842E00E945F3564
:1054800080912F0390913003079709F0D8C0809145
:105490004F0390E08C159D0509F4D1C09C2CC0925F
:1054A0003B0380914704811127C080EE9FEF9093CA
:1054B0005D0480935C0490935B0480935A04E12C18
:1054C000F12C0CE210E020E230E04CE350E063E726
:1054D00070E08AE494E00E949D1783E790E0909347
:1054E0005704809356048CE390E090935904809382
:1054F000580486E080935E0480914704813039F53A
:1055000080EE9FEF90935D0480935C0490935B0426
:1055100080935A04E12CF12C0CE210E029E130E0F8
:105520004CE450E06AE770E08AE494E00E949D1742
:105530008AE790E090935704809356048CE490E0BF
:10554000909359048093580485E080935E04809181
:105550004704823029F5B0925D04A0925C04B092B9
:105560005B04A0925A04E12CF12C04E510E020E445
:1055700030E044E150E067E370E08AE494E00E94A8
:105580009D1787E390E0909357048093560484E13D
:1055900090E090935904809358048CE080935E04CB
:1055A00098E0991206C066EF71E08AE494E00E94E8
:1055B000871480913B03873031F464E172E08AE420
:1055C00094E00E94871480913B03863031F461E5BA
:1055D00072E08AE494E00E94871480913B03853056
:1055E00031F463E572E08AE494E00E9487148091CC
:1055F0003B03843031F468E272E08AE494E00E9474
:10560000871480913B03833031F466E272E08AE4D0
:1056100094E00E94871480913B03823031F46CE364
:1056200072E08AE494E00E94871480913B03813009
:1056300031F464E272E08AE494E00E94871480917D
:105640002F03909130030897B1F580914E0390E0BD
:105650008C159D0581F1C0923A0380914704811118
:105660002AC080EE9FEF90935D0480935C0490933A
:105670005B0480935A04E12CF12C08E110E024E152
:1056800030E04CE350E06CE170E08AE494E00E948A
:105690009D178CE190E090935704809356048CE31F
:1056A00090E0909359048093580482E080935E04C4
:1056B0008C2D0E94C01A80912F039091300309977E
:1056C00009F091C18C2DC0924903109239031092B8
:1056D000380310923703109236031092350310925C
:1056E0003403803228F081E08093380380EE8C0D03
:1056F000803120F091E0909339038051883020F080
:1057000091E0909337038850843020F091E090939B
:1057100036038450823020F091E09093350382501C
:10572000882319F081E0809334038091470481112C
:105730005AC180913503813091F4C12C18EFD12EDC
:1057400002E4E02EF12C0FE510E022E430E041E429
:1057500050E063E370E080E590E00E948833809140
:105760003503811120C0C12CD12CA1E4EA2EF12CEB
:105770000EE510E021E430E040E450E064E370E046
:1057800080E590E00E948833B2E4EB2EF12C0FE527
:1057900010E022E430E041E450E063E370E080E5B3
:1057A00090E00E94311C8091360390914703981736
:1057B000C1F1813091F4C12CE8EFDE2EF6E4EF2E3A
:1057C000F12C0FE510E026E430E041E450E065E51F
:1057D00070E080E590E00E9488338091360381116B
:1057E00020C0C12CD12C67E4E62EF12C0EE510E090
:1057F00027E430E040E450E064E570E080E590E0CC
:105800000E94883376E4E72EF12C0FE510E026E4C1
:1058100030E041E450E065E570E080E590E00E9412
:10582000311CD0903703809148038D1509F46AC06C
:1058300081E0D8122BC0E12C58EFF52E07E010E0E4
:1058400020E130E048E250E06AE570E08CE390E06F
:105850000E94233384E490E090935704809356048D
:105860008EE590E09093590480935804D0925E04A2
:1058700010925D0410925C0410925B0410925A0422
:1058800061E172E08AE494E00E947314809137032E
:10589000811138C0E12CF12C07E010E020E130E06C
:1058A00048E250E06AE570E08CE390E00E94233328
:1058B0004FE1E42EF12C20E130E048E250E06AE5CF
:1058C00070E08CE390E00E94921B84E490E090935F
:1058D0005704809356048EE590E09093590480938A
:1058E000580481E080935E04B0925D04A0925C0451
:1058F000B0925B04A0925A0461E172E08AE494E001
:105900000E947314D0903403809145038D1509F4DF
:105910006AC091E0D9122BC0E12C38EFF32E07E0DA
:1059200010E020E130E048E250E06EE670E08CE309
:1059300090E00E9423338FE390E09093570480938C
:10594000560482E790E09093590480935804D092D3
:105950005E0410925D0410925C0410925B0410923D
:105960005A0466E172E08AE494E00E947314809124
:105970003403811138C0E12CF12C07E010E020E164
:1059800030E048E250E06EE670E08CE390E00E9488
:1059900023338FE390E0909357048093560482E77B
:1059A00090E0909359048093580481E080935E04C2
:1059B000B0925D04A0925C04B0925B04A0925A0481
:1059C00066E172E08AE494E00E9473142FE1E22E13
:1059D000F12C20E130E048E250E06EE670E08CE32C
:1059E00090E00E94921B80914704813009F040C2F0
:1059F00080913503909146039817C1F1813091F45D
:105A0000C12C88EFD82E91E3E92EF12C0BE210E0A7
:105A100021E330E04DE050E062E270E08CE190E0A4
:105A20000E94883380913503811120C0C12CD12C74
:105A300010E3E12EF12C0AE210E020E330E04CE02C
:105A400050E063E270E08CE190E00E94883301E373
:105A5000E02EF12C0BE210E021E330E04DE050E0CD
:105A600062E270E08CE190E00E94311C809136038C
:105A7000909147039817C1F1813091F4C12CA8EFA0
:105A8000DA2EB5E3EB2EF12C0BE210E025E330E04B
:105A90004DE050E064E470E08CE190E00E948833D7
:105AA00080913603811120C0C12CD12CE6E3EE2E6B
:105AB000F12C0AE210E026E330E04CE050E063E431
:105AC00070E08CE190E00E948833F5E3EF2EF12C3A
:105AD0000BE210E025E330E04DE050E064E470E0DC
:105AE0008CE190E00E94311CD090370380914803F4
:105AF0008D1509F46AC081E0D8122BC0E12C78EF33
:105B0000F72E07E010E020E130E04CE150E06CE4DB
:105B100070E080E090E00E94233383E090E0909377
:105B200057048093560480E590E090935904809345
:105B30005804D0925E0410925D0410925C0410929E
:105B40005B0410925A0461E172E08AE494E00E94DE
:105B5000731480913703811138C0E12CF12C07E0D8
:105B600010E020E130E04CE150E06CE470E080E0D7
:105B700090E00E9423336FE1E62EF12C20E130E02B
:105B80004CE150E06CE470E080E090E00E94921BF9
:105B900083E090E0909357048093560480E590E072
:105BA000909359048093580481E080935E04B092EE
:105BB0005D04A0925C04B0925B04A0925A0461E17F
:105BC00072E08AE494E00E947314D09034038091D0
:105BD00045038D1509F46AC091E0D9122BC0E12C60
:105BE00058EFF52E07E010E020E130E04CE150E006
:105BF0006CE470E08CE390E00E9423338FE390E04C
:105C0000909357048093560480E590E09093590454
:105C100080935804D0925E0410925D0410925C044C
:105C200010925B0410925A0465E572E08AE494E0F5
:105C30000E94731480913403811138C0E12CF12C3F
:105C400007E010E020E130E04CE150E06CE470E06F
:105C50008CE390E00E9423334FE1E42EF12C20E10D
:105C600030E04CE150E06CE470E08CE390E00E94A6
:105C7000921B8FE390E0909357048093560480E545
:105C800090E0909359048093580481E080935E04DF
:105C9000B0925D04A0925C04B0925B04A0925A049E
:105CA00065E572E08AE494E00E947314D0903903B1
:105CB000809133038D1509F46AC081E0D8122BC09E
:105CC000E12C38EFF32E07E010E020E130E04CE16A
:105CD00050E06CE470E08EE190E00E94233381E2BA
:105CE00090E0909357048093560480E590E0909361
:105CF000590480935804D0925E0410925D0410926F
:105D00005C0410925B0410925A046AE572E08AE423
:105D100094E00E94731480913903811138C0E12C02
:105D2000F12C07E010E020E130E04CE150E06CE4C1
:105D300070E08EE190E00E9423332FE1E22EF12CFF
:105D400020E130E04CE150E06CE470E08EE190E066
:105D50000E94921B81E290E0909357048093560436
:105D600080E590E0909359048093580481E08093FB
:105D70005E04B0925D04A0925C04B0925B04A092B9
:105D80005A046AE572E08AE494E00E947314D090A9
:105D90003803809132038D1509F46AC091E0D9125D
:105DA0002BC0E12C98EFF92E07E010E020E130E065
:105DB0004CE150E06CE470E08AE590E00E9423330F
:105DC0008DE590E0909357048093560480E590E031
:105DD0009093590480935804D0925E0410925D040D
:105DE00010925C0410925B0410925A046FE572E00A
:105DF0008AE494E00E94731480913803811138C0C2
:105E0000E12CF12C07E010E020E130E04CE150E023
:105E10006CE470E08AE590E00E9423338FE1E82E85
:105E2000F12C20E130E04CE150E06CE470E08AE5D8
:105E300090E00E94921B8DE590E090935704809330
:105E4000560480E590E0909359048093580481E0D3
:105E500080935E04B0925D04A0925C04B0925B04F7
:105E6000A0925A046FE572E08AE494E00E947314F1
:105E700080914704823009F05EC180913503909192
:105E800046039817C1F1813091F4C12CA8EFDA2EA6
:105E9000B2E4EB2EF12C03E210E022E430E045E026
:105EA00050E063E370E084E190E00E9488338091E9
:105EB0003503811120C0C12CD12CE1E4EE2EF12C50
:105EC00002E210E021E430E044E050E064E370E0FE
:105ED00084E190E00E948833F2E4EF2EF12C03E29B
:105EE00010E022E430E045E050E063E370E084E15C
:105EF00090E00E94311C80913603909147039817DF
:105F0000C1F1813091F4C12C68EFD62E76E4E72EF2
:105F1000F12C03E210E026E430E045E050E065E5D6
:105F200070E084E190E00E94883380913603811113
:105F300020C0C12CD12C47E4E42EF12C02E210E069
:105F400027E430E044E050E064E570E084E190E074
:105F50000E94883356E4E52EF12C03E210E026E49B
:105F600030E045E050E065E570E084E190E00E94BB
:105F7000311CD0903703809148038D1509F46AC015
:105F800081E0D8122BC0E12C38EFF32E07E010E0AF
:105F900020E130E048E250E06AE570E080E090E027
:105FA0000E94233384E490E0909357048093560436
:105FB0008EE590E09093590480935804D0925E044B
:105FC00010925D0410925C0410925B0410925A04CB
:105FD00061E172E08AE494E00E94731480913703D7
:105FE000811138C0E12CF12C07E010E020E130E015
:105FF00048E250E06AE570E080E090E00E942333E0
:106000002FE1E22EF12C20E130E048E250E06AE599
:1060100070E080E090E00E94921B88E090E0909316
:106020005704809356048EE590E090935904809332
:10603000580481E080935E04B0925D04A0925C04F9
:10604000B0925B04A0925A0461E172E08AE494E0A9
:106050000E947314D0903403809145038D1509F488
:106060006AC091E0D9122BC0E12C98EFF92E07E01D
:1060700010E020E130E048E250E06EE670E080E0C1
:1060800090E00E94233383E090E090935704809344
:10609000560482E790E09093590480935804D0927C
:1060A0005E0410925D0410925C0410925B041092E6
:1060B0005A0466E172E08AE494E00E9473148091CD
:1060C0003403811138C0E12CF12C07E010E020E10D
:1060D00030E048E250E06EE670E080E090E00E9440
:1060E000233383E090E0909357048093560482E733
:1060F00090E0909359048093580481E080935E046B
:10610000B0925D04A0925C04B0925B04A0925A0429
:1061100066E172E08AE494E00E9473148FE1E82E55
:10612000F12C20E130E048E250E06EE670E080E0E3
:1061300090E00E94921B80913103809349038091EB
:106140003903809333038091380380933203809125
:1061500037038093480380913603809347038091EF
:1061600035038093460380913403809345038091E7
:106170002F03909130030C9709F450C040912A03EB
:1061800050912B0360912C0370912D032FB7F8943D
:106190008091260390912703A0912803B0912903B1
:1061A0002FBF481759076A077B07C0F10E94C31227
:1061B0000C94491D87E290E00C9401248FE490E058
:1061C0000C94532489E090E09093570480935604F4
:1061D0008DE690E0909359048093580490925D046A
:1061E00080925C0490925B0480925A040C94C627BF
:1061F00089E090E090935704809356048EE090E0FD
:10620000909359048093580490925D0480925C04AA
:1062100090925B0480925A040C94352810923003BB
:1062200010922F0380914403809354038091430381
:1062300080935303809142038093520380914103E2
:1062400080935103809140038093500380913B03DE
:1062500080934F0380913A0380934E0380913C03D7
:1062600090913D03A0913E03B0913F0380934A0378
:1062700090934B03A0934C03B0934D038091000186
:1062800090910101909303018093020164E672E012
:1062900088EA93E00E9487140E94210E87CF87E44A
:1062A00091E090937A048093790489E794E00C94C8
:1062B00074161092AB031092AA0388EE93E0A0E04C
:1062C000B0E08093AC039093AD03A093AE03B09382
:1062D000AF0329E031E03093A9032093A80325EC14
:1062E00030E03093B5032093B40324EC30E03093D6
:1062F000B7032093B60320EC30E03093B90320932A
:10630000B80321EC30E03093BB032093BA0322ECB6
:1063100030E03093BD032093BC0326EC30E0309393
:10632000BF032093BE031092C1031092C2031092C8
:10633000C3031092C40320E5209345041092460441
:1063400010927C0410927B0480937D0490937E04D1
:10635000A0937F04B093800487E491E090937A0443
:10636000809379041092900410928F0410929204FA
:106370001092910410929404109293041092960437
:1063800010929504609197046E7F6D7F60939704DF
:106390006695617081E0682783E00E940A1561E0DC
:1063A00083E00E943A15E5E7F0E1E491E093890487
:1063B000E1E6F0E1E491F0E0EE0FFF1FE65BFF4E57
:1063C0008591949190938B0480938A0460E082E09D
:1063D0000E943A158091970481FD04C061E082E03B
:1063E0000E940A1582E080938504E4E7F0E1E491DD
:1063F000E0938604E0E6F0E1E491F0E0EE0FFF1FA9
:10640000EC5AFF4E85919491909388048093870471
:1064100010924D0410924C0420E830E030934F0469
:1064200020934E0480EA90E09093510480935004AE
:106430003093530420935204909355048093540452
:1064400010925F041092570410925604109259044F
:106450001092580481E080935E042FEF3FEF309359
:106460005D0420935C0430935B0420935A04809372
:1064700060041092610410926304109262042BE194
:1064800031E030934B0420934A049AE090936E04D9
:1064900098E090936F0499E0909370048093650462
:1064A000109272041092710480E090E00E943D36D8
:1064B0008093490481E090E00E943D368093480437
:1064C00082E090E00E943D368093470408952F9229
:1064D0003F924F925F926F927F928F929F92AF9274
:1064E000BF92CF92DF92EF92FF920F931F93CF93C1
:1064F000DF9300D000D000D0CDB7DEB75C014B01F8
:106500005E834D83280181E090E03C01641A750AA6
:10651000CA01919581959109AC01440F551F5A8389
:1065200049831801CC24C394D12C522F51705B8322
:1065300022702C83C60101972D813E81821793071B
:106540000CF068C077FC0CC08D819E8101979E8302
:106550008D83E981FA813296FA83E9836E0E7F1E7C
:10656000C601880F991F0196680E791EFB81FF23D3
:1065700019F12D813E81220F331F2F5F3F4F240DD4
:10658000351D8701A4018D819E81481B590BB601E1
:106590006A0D7B1D8AE494E00E945B0D91012D5FE2
:1065A0003F4FA4014C195D096D817E816A0D7B1DF1
:1065B0008AE494E00E945B0D9C81992321F12D8156
:1065C0003E81220F331F2F5F3F4F240D351D870162
:1065D000A401ED81FE814E1B5F0BB5016C197D0995
:1065E0008AE494E00E945B0D91012D5F3F4FA4016E
:1065F0004C195D09B5018D819E81681B790B8AE478
:1066000094E00E945B0D9FEFC91AD90AE2E02E0EBA
:10661000311C90CF26960FB6F894DEBF0FBECDBFCB
:10662000DF91CF911F910F91FF90EF90DF90CF906E
:10663000BF90AF909F908F907F906F905F904F90A2
:106640003F902F9008952F923F924F925F926F92BA
:106650007F928F929F92AF92BF92CF92DF92EF92F2
:10666000FF920F931F93CF93DF9300D000D0CDB74D
:10667000DEB72C015B011A013901680188279927CF
:10668000801B910B9C01220F331F3C832B83C20183
:10669000800F911F9A838983240F351F8301AB01DB
:1066A000BC018AE494E00E943F0DEB81FC816E0EF8
:1066B0007F1EF1E06F1A7108AC0CBD1C420C531C1C
:1066C000C2018C199D09830121E0A601B501019742
:1066D0000E94673222E0A601B50189819A810E9459
:1066E00067320F900F900F900F90DF91CF911F9115
:1066F0000F91FF90EF90DF90CF90BF90AF909F9061
:106700008F907F906F905F904F903F902F90089563
:106710002F923F924F925F926F927F928F929F92B1
:10672000AF92BF92CF92DF92EF92FF920F931F939F
:10673000CF93DF93CDB7DEB7AC970FB6F894DEBF3B
:106740000FBECDBF9CA78BA73B015A014901B801E1
:10675000DC8ACB8A2615370584F4892DE614F704E4
:106760000CF08BC147017301622E782E8B2D5801DE
:106770006BA57CA54BA78CA70DC0E216F306C4F44D
:10678000982D892D4701E92EF82E9A2D8B2D5B012E
:10679000692F782F861497045CF4962D872D340189
:1067A000892E982E9BA58CA5BCA6ABA6A92EB82E8B
:1067B0006E147F0449F52BA53CA5A216B3065CF028
:1067C0009BA58CA52A153B0514F49A2D8B2DABA403
:1067D000BCA49BA78CA76A157B0544F04BA55CA5C0
:1067E0004617570714F47CA76BA7B5012BA53CA54A
:1067F000261B370B2F5F3F4F0B891C89A3018AE4AF
:1068000094E00E944F0D42C1C501ABA5BCA58A1BF7
:106810009B0B940126193709FB01EA1BFB0BFC8338
:10682000EB83A7014619570958874F83DB01AA1943
:10683000BB09BC87AB87F701E819F909FE8BED8B23
:106840008E149F0431F0A401415051095A8F498F91
:1068500002C09A8E898E6301212C312C21011F8662
:10686000188A198A1A8AA901330F660B770B4B8F86
:106870005C8F6D8F7E8F2F813885032E000C440B2B
:10688000550B2F8F38A349A35AA3AC01990F660B60
:10689000770B4BA35CA36DA37EA36B817C81072E3A
:1068A000000C880B990B6FA378A789A79AA7A98DCD
:1068B000BA8DAC15BD050CF451C06F8578898989F6
:1068C0009A892B8D3C8D4D8D5E8D0E94CC388BA589
:1068D0009CA5820F931F9A838983C201B1012F8DDA
:1068E00038A149A15AA10E94CC38ABA5BCA52A0F5A
:1068F0003B1F4F85588969897A898BA19CA1ADA1DD
:10690000BEA1480F591F6A1F7B1F4F87588B698B89
:106910007A8B4FA158A569A57AA5240E351E461E6F
:10692000571E69817A812617370734F499818A8145
:106930003A832983292F382F89819A81281B390B83
:106940002F5F3F4F0B891C89A601BC018AE494E0AC
:106950000E944F0D9FEFC91AD90AA9CFC601881905
:106960009909EB85FC85E89F1001E99F300CF89FA1
:10697000300C1124032C000C44085508C60186195C
:1069800097092B813C81289F3001299F700C389FEB
:10699000700C1124072C000C880899084D895E8919
:1069A000052E000C660B770B4D8B5E8B6F8B788FF3
:1069B0006F817885072E000C880B990B6F83788781
:1069C00089879A87CF01092E000CAA0BBB0B8B87F6
:1069D0009C87AD87BE87032E000C440B550B2B8381
:1069E0003C834D835E83EC14FD040CF44FC0C20164
:1069F000B1012D893E894F89588D0E94CC38B5014F
:106A0000620F731F7A836983C401B3012F813885B4
:106A100049855A850E94CC388BA59CA5280F391F23
:106A20004B855C856D857E85240E351E461E571E62
:106A30006B817C818D819E81660E771E881E991EDA
:106A400089819A812817390734F499818A813A8398
:106A50002983292F382FA981BA812A1B3B0B2F5F4D
:106A60003F4F0B891C89A601BD018AE494E00E9476
:106A70004F0DBFEFCB1ADB0AB6CF4301622E782E43
:106A80008B2DABA4BCA44BA78CA792CEAC960FB613
:106A9000F894DEBF0FBECDBFDF91CF911F910F9154
:106AA000FF90EF90DF90CF90BF90AF909F908F902E
:106AB0007F906F905F904F903F902F9008954F92EE
:106AC0005F926F927F928F929F92AF92BF92CF927E
:106AD000DF92EF92FF926B017C01B42E9B01AC011F
:106AE0000E949138882319F06AE173E027C02601DB
:106AF0003701E89477F82FEF3FEF4FE75FE7C301E7
:106B0000B2010E94913881110DC02FEF3FEF4FE786
:106B10005FE7C301B2010E94C03618161CF46EE193
:106B200073E00CC02FEF3FEF4FE75FE4C701B60102
:106B30000E941F38181694F462E273E08AE494E02D
:106B4000FF90EF90DF90CF90BF90AF909F908F908D
:106B50007F906F905F904F900C9415142FEF3FEF44
:106B60004FE75FECC701B6010E94C03687FDE4CF56
:106B700020E030E0A901C701B6010E94C03687FFBE
:106B80000BC06DE28AE494E00E940E144C01F7FA07
:106B9000F094F7F8F09402C0812C912CA12C60E0C5
:106BA00070E080E09FE3AB1441F020E030E040E291
:106BB00051E40E94C536A394F6CF9B01AC01C701F6
:106BC000B6010E9454362B013C010E943E376B01F6
:106BD0007C010E946D379B01AC01C301B2010E9490
:106BE00053362B013C012AE0B701A6018AE494E068
:106BF0000E942A147C01E80CF91CBB2039F06EE2DB
:106C00008AE494E00E940E14E80EF91EDB2CDD20CD
:106C100031F120E030E040E251E4C301B2010E94D2
:106C200024382B013C010E943E374B01A12CB12C92
:106C30002AE0B501A4018AE494E00E942A14E80E37
:106C4000F91EC501B4010E946D379B01AC01C3015F
:106C5000B2010E9453362B013C01DA94D8CFC70110
:106C6000FF90EF90DF90CF90BF90AF909F908F906C
:106C70007F906F905F904F900895F999FECF92BDED
:106C800081BDF89A992780B50895262FF999FECFEE
:106C90001FBA92BD81BD20BD0FB6F894FA9AF99A39
:106CA0000FBE019608955058BB27AA270E946B3645
:106CB0000C94E5370E94D73738F00E94DE3720F079
:106CC00039F49F3F19F426F40C94D4370EF4E09570
:106CD000E7FB0C94CE37E92F0E94F63758F3BA172A
:106CE000620773078407950720F079F4A6F50C94E2
:106CF00018380EF4E0950B2EBA2FA02D0B01B90118
:106D000090010C01CA01A0011124FF27591B99F021
:106D1000593F50F4503E68F11A16F040A22F232F2D
:106D2000342F4427585FF3CF469537952795A7957D
:106D3000F0405395C9F77EF41F16BA0B620B730B24
:106D4000840BBAF09150A1F0FF0FBB1F661F771F95
:106D5000881FC2F70EC0BA0F621F731F841F48F44A
:106D6000879577956795B795F7959E3F08F0B0CFD3
:106D70009395880F08F09927EE0F979587950895BA
:106D80000E94AA3708F481E008950E94D9360C9435
:106D9000E5370E94DE3758F00E94D73740F029F4DB
:106DA0005F3F29F00C94CE3751110C9419380C9494
:106DB000D4370E94F63768F39923B1F3552391F342
:106DC000951B550BBB27AA2762177307840738F05A
:106DD0009F5F5F4F220F331F441FAA1FA9F335D0B7
:106DE0000E2E3AF0E0E832D091505040E695001C6B
:106DF000CAF72BD0FE2F29D0660F771F881FBB1F25
:106E0000261737074807AB07B0E809F0BB0B802D02
:106E1000BF01FF2793585F4F3AF09E3F510578F02E
:106E20000C94CE370C9419385F3FE4F3983ED4F3BA
:106E3000869577956795B795F7959F5FC9F7880F02
:106E4000911D9695879597F90895E1E0660F771F54
:106E5000881FBB1F621773078407BA0720F0621BE5
:106E6000730B840BBA0BEE1F88F7E09508950E9410
:106E70003E376894B1110C94193808950E94FE377A
:106E800088F09F5798F0B92F9927B751B0F0E1F0EB
:106E9000660F771F881F991F1AF0BA95C9F714C09B
:106EA000B13091F00E941838B1E008950C94183870
:106EB000672F782F8827B85F39F0B93FCCF38695D4
:106EC00077956795B395D9F73EF490958095709531
:106ED00061957F4F8F4F9F4F0895E89409C097FBAE
:106EE0003EF490958095709561957F4F8F4F9F4FA1
:106EF0009923A9F0F92F96E9BB279395F6958795E5
:106F000077956795B795F111F8CFFAF4BB0F11F4A7
:106F100060FF1BC06F5F7F4F8F4F9F4F16C088234E
:106F200011F096E911C0772321F09EE8872F762F84
:106F300005C0662371F096E8862F70E060E02AF0C5
:106F40009A95660F771F881FDAF7880F96958795B1
:106F500097F90895990F0008550FAA0BE0E8FEEF86
:106F600016161706E807F907C0F012161306E4070D
:106F7000F50798F0621B730B840B950B39F40A2606
:106F800061F0232B242B252B21F408950A2609F4E4
:106F9000A140A6958FEF811D811D089597F99F67E8
:106FA00080E870E060E008959FEF80EC0895002491
:106FB0000A941616170618060906089500240A945E
:106FC00012161306140605060895092E0394000CE4
:106FD00011F4882352F0BB0F40F4BF2B11F460FF73
:106FE00004C06F5F7F4F8F4F9F4F089557FD90589C
:106FF000440F551F59F05F3F71F04795880F97FB7D
:10700000991F61F09F3F79F0879508951216130636
:107010001406551FF2CF4695F1DF08C01616170665
:107020001806991FF1CF869571056105089408959A
:10703000E894BB2766277727CB0197F908950E942C
:10704000AA3708F48FEF08950E9437380C94E5377B
:107050000E94D73738F00E94DE3720F0952311F0D8
:107060000C94CE370C94D43711240C9419380E9408
:10707000F63770F3959FC1F3950F50E0551F629F4F
:10708000F001729FBB27F00DB11D639FAA27F00D81
:10709000B11DAA1F649F6627B00DA11D661F829FA8
:1070A0002227B00DA11D621F739FB00DA11D621F8D
:1070B000839FA00D611D221F749F3327A00D611DAA
:1070C000231F849F600D211D822F762F6A2F11248C
:1070D0009F5750409AF0F1F088234AF0EE0FFF1FBF
:1070E000BB1F661F771F881F91505040A9F79E3F16
:1070F000510580F00C94CE370C9419385F3FE4F3BF
:10710000983ED4F3869577956795B795F795E7956B
:107110009F5FC1F7FE2B880F911D9695879597F974
:1071200008950E94AA37880B990B089597FB072EA4
:1071300016F4009407D077FD09D00E94EB3807FCC5
:1071400005D03EF4909581959F4F08957095619577
:107150007F4F0895A1E21A2EAA1BBB1BFD010DC093
:10716000AA1FBB1FEE1FFF1FA217B307E407F507F7
:1071700020F0A21BB30BE40BF50B661F771F881FD3
:10718000991F1A9469F760957095809590959B0169
:10719000AC01BD01CF010895052E97FB1EF40094AC
:1071A0000E94E33857FD07D00E94AA3807FC03D09D
:1071B0004EF40C94E33850954095309521953F4F0F
:1071C0004F4F5F4F089590958095709561957F4FD3
:1071D0008F4F9F4F0895AA1BBB1B51E107C0AA1FE9
:1071E000BB1FA617B70710F0A61BB70B881F991F68
:1071F0005A95A9F780959095BC01CD010895EE0FA1
:10720000FF1F0590F491E02D099481E090E0F8943F
:107210000C940A3918E0C4E4D8E004C0FE010E94CE
:0E722000FF382196C534D107C9F7F894FFCF87
:10722E000100010001000000005A12C711F211A165
:10723E0012231201121512000000009B0AC7111A28
:10724E000E190ED5186E0D670D3F0D5B0D4F0D6FA0
:10725E000D3E0D0417FD16761817189D17C113D085
:10726E000B710B000000003413C7111A0E33138874
:10727E0013A0131B13536F667477617265205365E9
:10728E007269616C20506F7274204F70656E656408
:10729E0000536176696E672073657474696E6773E7
:1072AE002E2E2E2000536176696E672073657474DE
:1072BE00696E677300202D20446F6E652100646136
:1072CE00796C75782073657474696E67733A2000F3
:1072DE006E696768746C75782073657474696E670F
:1072EE00733A200053637265656E2030005450531C
:1072FE000030302020250042415400202020202044
:10730E0056004F494C002020202027430052504D5C
:10731E00003030004D41500053686966746572004C
:10732E0053656C0043757200202020006B6D002F9A
:10733E00004C6F7752004C6F636B55700053637245
:10734E0065656E203100330034003600370038009A
:10735E006B6D2F680053637265656E203200093ABB
:10736E00000D0A004F696C202743004C4F57212116
:10737E00004E0044004C6B5570004F447276003244
:10738E0047725300200950617373204D6164653A52
:10739E00200053656E64696E6720323532202D00F1
:1073AE0053706974726F6E6963730053656E6469AE
:1073BE006E6720323535003A202009004E6F496E37
:1073CE00697400454355005443550043414D0054E4
:1073DE0048785700454D5500546974616E005665E6
:1073EE006E7573004D65726375727900506C7574AD
:1073FE006F004D65726375727932004E65707475EB
:10740E006E65004E657074756E65320020762E00C6
:10741E00446973706C617920556E697420762E31D3
:10742E0035006461796C75783A00206E696768740E
:10743E006C75783A0020280029006E616E00696E26
:06744E0066006F76660087
:00000001FF
